Open Watcom Linker Version 1.0
Portions Copyright (c) 1985-2002 Sybase, Inc. All Rights Reserved.
Created on:       03/04/01 18:15:42
Executable Image: duke3d.exe
creating a DOS/4G executable


                        +------------+
                        |   Groups   |
                        +------------+

Group                           Address              Size
=====                           =======              ====

DGROUP                          0003:00000000        002315a0



                        +--------------+
                        |   Segments   |
                        +--------------+

Segment                Class          Group          Address         Size
=======                =====          =====          =======         ====

BEGTEXT                CODE           AUTO           0001:00000000   00000010
_TEXT                  CODE           AUTO           0001:00000010   000a2d90
CODE                   CODE           AUTO           0001:000a2da0   00001795
TEXT                                  AUTO           0002:00000000   0000005d
digital11_DATA         FAR_DATA       AUTO           0002:0000005d   00000000
gf1mem11_DATA          FAR_DATA       AUTO           0002:0000005d   00000000
gf1init11_DATA         FAR_DATA       AUTO           0002:0000005d   00000000
gf1patch11_DATA        FAR_DATA       AUTO           0002:0000005d   00000000
gf1note11_DATA         FAR_DATA       AUTO           0002:0000005d   00000000
gf1isr11_DATA          FAR_DATA       AUTO           0002:0000005d   00000000
gf1addr11_DATA         FAR_DATA       AUTO           0002:0000005d   00000000
divisor11_DATA         FAR_DATA       AUTO           0002:0000005d   00000000
gf1dma11_DATA          FAR_DATA       AUTO           0002:0000005d   00000000
gf1voice11_DATA        FAR_DATA       AUTO           0002:0000005d   00000000
gf1dram11_DATA         FAR_DATA       AUTO           0002:0000005d   00000000
os11_DATA              FAR_DATA       AUTO           0002:0000005d   00000000
gf1wisr11_DATA         FAR_DATA       AUTO           0002:0000005d   00000000
gf1detct11_DATA        FAR_DATA       AUTO           0002:0000005d   00000000
gf1wave11_DATA         FAR_DATA       AUTO           0002:0000005d   00000000
timer11_DATA           FAR_DATA       AUTO           0002:0000005d   00000000
_NULL                  BEGDATA        DGROUP         0003:00000000   00000004
_AFTERNULL             BEGDATA        DGROUP         0003:00000004   00000000
CONST                  DATA           DGROUP         0003:00000004   0000679c
CONST2                 DATA           DGROUP         0003:000067a0   000002c9
_DATA                  DATA           DGROUP         0003:00006a70   0000a60c
TIB                    DATA           DGROUP         0003:0001107c   00000000
TI                     DATA           DGROUP         0003:0001107c   00000000
TIE                    DATA           DGROUP         0003:0001107c   00000000
XIB                    DATA           DGROUP         0003:0001107c   00000000
XI                     DATA           DGROUP         0003:0001107c   00000048
XIE                    DATA           DGROUP         0003:000110c4   00000000
YIB                    DATA           DGROUP         0003:000110c4   00000000
YI                     DATA           DGROUP         0003:000110c4   0000002a
YIE                    DATA           DGROUP         0003:000110ee   00000000
DATA                   DATA           DGROUP         0003:000110ee   00000000
_GF1INITS              DATA           DGROUP         0003:000110ee   00000000
_GF1INIT               DATA           DGROUP         0003:000110ee   00000024
_GF1INITE              DATA           DGROUP         0003:00011112   00000000
_BSS                   BSS            DGROUP         0003:00011120   00209c80
STACK                  STACK          DGROUP         0003:0021ada0   00016800


                        +----------------+
                        |   Memory Map   |
                        +----------------+

* = unreferenced symbol
+ = symbol only referenced locally

Address        Symbol
=======        ======

Module: game.obj(H:\Games\duke3d\source\game.c)
0003:00011120+ _tempsectorz
0003:00012120+ _tempsectorpicnum
0003:00013160+ _user_quote
0003:00013360+ _recbuf
0003:000133b0+ _user_quote_time
0003:000133b8  _titlepal
0003:000136b8  _waterpal
0003:000139b8  _drealms
0003:00013cb8  _endingpal
0003:00013fb8  _slimepal
0003:000142b8+ _nonsharedtimer
0003:000142bc+ _quotebotgoal
0003:000142c0+ _quotebot
0003:000142c4+ _recfilep
0003:000142c8+ _rtsptr
0003:000142cc+ _totalreccnt
0003:000142d0  _tempwallptr
0003:00006a70  _cameradist
0003:00006a74  _cameraclock
0003:00006a78  _eightytwofifty
0003:00006a7c+ _CommandSoundToggleOff
0003:00006a80+ _CommandMusicToggleOff
0003:00006a84+ _confilename
0003:00006b04  _boardfilename
0003:00006b84+ _firstdemofile
0003:00006bd4+ _debug_on
0003:00006bd5  _actor_tog
0003:00006bd6+ _memorycheckoveride
0003:00006bd8+ _frecfilep
0003:00006bdc+ _sendmessagecommand
0003:00006be0+ _TimerPtr
0003:00006be8  _inputloc
0003:00006bf0+ _cheatquotes
0001:000001d0+ timerhandler_
0001:000001e0+ inittimer_
0001:00000210  uninittimer_
0001:00000250  gametext_
0001:00000370  gametextpal_
0001:00000490* gametextpart_
0001:000005f0  minitext_
0001:00000690+ minitextshade_
0001:00000730* gamenumber_
0001:00000770+ allowtimetocorrecterrorswhenquitting_
0001:00000800+ adduserquote_
0001:000008a0  getpackets_
0001:00001900  faketimerhandler_
0001:000028b0+ caches_
0001:00002990+ checksync_
0001:00002b40  check_fta_sounds_
0001:00002db0  inventory_
0001:00002df0  badguy_
0001:00002f70  badguypic_
0001:000030f0  myos_
0001:000031a0  myospal_
0001:00003210+ invennum_
0001:00003400+ weaponnum_
0001:000036c0+ weaponnum999_
0001:00003ac0+ weapon_amounts_
0001:000042a0+ digitalnumber_
0001:000043a0+ displayinventory_
0001:00004780  displayfragbar_
0001:000049e0+ coolgaugetext_
0001:00005ac0+ tics_
0001:00005b50+ coords_
0001:00005e30+ operatefta_
0001:000060a0  FTA_
0001:00006110* showtwoscreens_
0001:00006120+ binscreen_
0001:00006160  gameexit_
0001:00006280  strget_
0001:00006480+ typemode_
0001:00006920+ moveclouds_
0001:00006a30+ displayrest_
0001:00007230+ updatesectorz_
0001:00007390+ view_
0001:000076d0  drawbackground_
0001:00007b60+ SE40_Draw_
0001:00007f80+ se40code_
0001:00008020  displayrooms_
0001:00008c20  LocateTheLocator_
0001:00008c70  EGS_
0001:00008ec0  wallswitchcheck_
0001:00009080  spawn_
0001:0000d740  animatesprites_
0001:0000f5f0+ cheats_
0001:00010480+ nonsharedkeys_
0001:000116b0+ comlinehelp_
0001:000118e0+ checkcommandline_
0001:00012030+ printstr_
0001:00012080+ Logo_
0001:00012690+ loadtmb_
0001:000126e0+ Shutdown_
0001:00012710+ compilecons_
0001:00012770+ Startup_
0001:000128a0  sendscore_
0001:000128e0+ getnames_
0001:00012ae0* writestring_
0001:00012b30* testcd_
0001:00012c40+ copyprotect_
0001:00012c50  main_
0001:00013380+ opendemoread_
0001:00013620  opendemowrite_
0001:00013840+ record_
0001:00013940  closedemowrite_
0001:000139e0+ playback_
0001:00013f40+ moveloop_
0001:00014010+ fakedomovethingscorrect_
0001:000141e0+ fakedomovethings_
0001:00015390+ domovethings_
0001:00015a50* doorders_
0001:00015d10  dobonus_
0001:000174d0+ cameratext_
0001:000176c0* vglass_
0001:000177b0  lotsofglass_
0001:00017a20  spriteglass_
0001:00017af0  ceilingglass_
0001:00017c30  lotsofcolourglass_
0001:00017e90+ SetupGameButtons_
0001:00018100+ GetTime_
0001:00018110+ CenterCenter_
0001:00018120+ UpperLeft_
0001:00018130+ LowerRight_
0001:00018140+ CenterThrottle_
0001:00018150+ CenterRudder_
0003:00006de0+ _which_demo
0003:00006de1+ _in_menu
0003:000142dc+ _cheatbuf
0003:000142e6+ _cheatbuflen
0003:000142e7+ _cp
0003:000142e8+ _qe
0003:000142e9+ _nomorelogohack
0003:000142ea+ _playerswhenstarted
0003:000142eb  _restorepalette
0003:000142ec  _screencapt
Module: actors.obj(H:\Games\duke3d\source\actors.c)
0001:00018180  updateinterpolations_
0001:000181b0  setinterpolation_
0001:00018200  stopinterpolation_
0001:00018280  dointerpolations_
0001:000182f0  restoreinterpolations_
0001:00018320  ceilingspace_
0001:00018370  floorspace_
0001:000183c0  addammo_
0001:00018430  addweapon_
0001:00018500  checkavailinven_
0001:00018590  checkavailweapon_
0001:000186f0  ifsquished_
0001:00018840  hitradius_
0001:000191e0  movesprite_
0001:000197a0  ssp_
0001:00019820  insertspriteq_
0001:000198c0  lotsofmoney_
0001:00019940  lotsofmail_
0001:000199c0  lotsofpaper_
0001:00019a40  guts_
0001:00019be0+ gutsdir_
0001:00019cf0  setsectinterpolate_
0001:00019dc0* clearsectinterpolate_
0001:00019e70+ ms_
0001:00019fa0  movefta_
0001:0001a2f0+ ifhitsectors_
0001:0001a330  ifhitbyweapon_
0001:0001a700  movecyclers_
0001:0001a810  movedummyplayers_
0001:0001a9e0  moveplayers_
0001:0001adc0  movefx_
0001:0001b210  movefallers_
0001:0001b580  movestandables_
0001:0001d4a0+ bounce_
0001:0001d6c0  moveweapons_
0001:0001e570  movetransports_
0001:0001f5c0  moveactors_
0001:00022640  moveexplosions_
0001:00023770  moveeffectors_
0003:000142f8  _otherp
Module: gamedef.obj(H:\Games\duke3d\source\gamedef.c)
0001:00028c60  getincangle_
0001:00028cb0+ ispecial_
0001:00028ce0+ isaltok_
0001:00028d20  getglobalz_
0001:00028fd0  makeitfall_
0001:000291e0+ getlabel_
0001:00029290+ keyword_
0001:00029310+ transword_
0001:00029530+ transnum_
0001:00029950+ parsecommand_
0001:0002b3d0+ passone_
0001:0002b400+ copydefaultcons_
0001:0002b4b0  loadefs_
0001:0002b7e0+ dodge_
0001:0002b940  furthestangle_
0001:0002ba80+ furthestcanseepoint_
0001:0002bc40+ alterang_
0001:0002bf30+ move_
0001:0002c850+ parseifelse_
0001:0002caa0+ parse_
0001:00030260  execute_
0003:00006de4+ _keyw
0003:00006fa4+ _defaultcons
Module: global.obj(H:\Games\duke3d\source\global.c)
0003:00014330  _bakipos
0003:00016330  _clouds
0003:00016430  _cloudy
0003:00016530  _cloudx
0003:00016630  _oldipos
0003:00018630  _myminlag
0003:00018670  _curipos
0003:0001a670  _syncval
0003:0001b670  _syncvalhead
0003:0001b6b0  _frags
0003:0001b8b0  _myzbak
0003:0001bcb0  _myxbak
0003:0001c0b0  _myybak
0003:0001c4b0  _myangbak
0003:0001c6b0  _myhorizbak
0003:0001cab0  _level_file_names
0003:0001e0b0  _betaname
0003:0001e100  _animatesect
0003:0001e180  _designertime
0003:0001e230  _mirrorsector
0003:0001e2b0  _soundsiz
0003:0001e9b8  _mirrorwall
0003:0001ea38  _partime
0003:0001eae8  _animateptr
0003:0001ebe8  _movefifoend
0003:0001ec28  _animatevel
0003:0001ed28  _animategoal
0003:0001ee28  _hittype
0003:00066e28  _actortype
0003:00068628  _script
0003:0007c5d8  _actorscrptr
0003:000825d8  _spriteq
0003:00082dd8  _Sound
0003:000849f8  _ud
0003:00085338  _buf
0003:00085388  _max_ammo_amount
0003:000853b8  _playerquitflag
0003:000853c8  _playerreadyflag
0003:000853d8  _SoundOwner
0003:00088c18  _po
0003:00088d18  _ps
0003:0008c658  _fta_quotes
0003:0008f658  _animwall
0003:00090658  _packbuf
0003:00090898  _cyclers
0003:00091498  _tempbuf
0003:00091c98  _myname
0003:00091cb8  _MusicPtr
0003:000a35f8  _msy
0003:000a55f8  _msx
0003:000a75f8  _recsync
0003:000aec18  _inputfifo
0003:000bac18  _sync
0003:000bacd8  _shrinkerblastradius
0003:000bacdc  _bouncemineblastradius
0003:000bace0  _mymaxlag
0003:000bace4  _otherminlag
0003:000bace8  _tripbombblastradius
0003:000bacec  _seenineblastradius
0003:000bacf0  _morterblastradius
0003:000bacf4  _syncvaltail
0003:000bacf8  _rpgblastradius
0003:000bacfc  _pipebombblastradius
0003:000bad00  _show_shareware
0003:000bad04  _syncvaltottail
0003:000bad08  _myzvel
0003:000bad0c  _myyvel
0003:000bad10  _myz
0003:000bad14  _omyz
0003:000bad18  _fakemovefifoplc
0003:000bad1c  _myxvel
0003:000bad20  _myy
0003:000bad24  _myx
0003:000bad28  _omyx
0003:000bad2c  _omyy
0003:000bad30  _neartaghitdist
0003:000bad34* _checksume
0003:000bad38  _svel
0003:000bad3c  _vel
0003:000bad40  _horiz
0003:000bad44  _soundpe
0003:000bb0c8  _soundps
0003:000bb44c  _volume_names
0003:000bb4d0  _angvel
0003:000bb4d4  _movefifoplc
0003:000bb4d8  _level_names
0003:000bba84  _soundvo
0003:000bbe08  _avgbits
0003:000bbe0c  _current_menu
0003:000bbe10  _ototalclock
0003:000bbe14  _avgsvel
0003:000bbe18  _avgavel
0003:000bbe1c  _avghorz
0003:000bbe20  _groupfile
0003:000bbe24  _animatecnt
0003:000bbe28  _lockclock
0003:000bbe2c  _insptr
0003:000bbe30* _music_pointer
0003:000bbe34  _music_fn
0003:000bc070  _labelcode
0003:000bc074  _sounds
0003:000bd910  _avgfvel
0003:000bd914  _labelcnt
0003:000bd918  _env_music_fn
0003:000bd94c  _loc
0003:000bd958  _parsing_actor
0003:000bd95c  _label
0003:000bd960  _scriptptr
0003:000bd964  _textptr
0003:000bd968  _impact_damage
0003:000bd96c* _device
0003:000bd978  _mymembuf
0003:000bd97c  _max_armour_amount
0003:000bd980  _gc
0003:000bd984  _movefifosendplc
0003:000bd988  _max_player_health
0003:000bd98c  _fricyv
0003:000bd990  _fricxv
0003:000bd99c  _sbar
0003:000bda02  _soundm
0003:000bdbc4  _soundpr
0003:000bdd86* _title_zoom
0003:000bdd88  _numclouds
0003:000bdd8a  _myhoriz
0003:000bdd8c  _omyhoriz
0003:000bdd8e  _myhorizoff
0003:000bdd90  _mycursectnum
0003:000bdd92  _myjumpingcounter
0003:000bdd94  _myang
0003:000bdd96  _omyang
0003:000bdd98  _omyhorizoff
0003:000bdd9a  _neartagsprite
0003:000bdd9c  _mirrorcnt
0003:000bdd9e  _neartagsector
0003:000bdda0  _screenpeek
0003:000bdda2  _neartagwall
0003:000bdda4  _camsprite
0003:000bdda6  _global_random
0003:000bdda8* _moustat
0003:000bddaa  _spriteqloc
0003:000bddac  _numcyclers
0003:000bddae  _numanimwalls
0003:000bddb0  _skill_names
0003:000bde55  _typebuf
0003:000bde7e  _everyothertime
0003:000bde7f  _multiwho
0003:000bde80  _lasermode
0003:000bde81  _multiflag
0003:000bde82  _syncstat
0003:000bde83  _camerashitable
0003:000bde84  _pub
0003:000bde85  _pus
0003:000bde86  _multiwhat
0003:000bde87  _multipos
0003:000bde88  _myreturntocenter
0003:000bde89  _myhardlanding
0003:000bde8a  _myjumpingtoggle
0003:000bde8b  _myonground
0003:000bde8c  _earthquaketime
0003:000bde8d  _loadfromgrouponly
0003:000bde8e  _rtsplaying
0003:000bde8f  _display_mirror
0003:000bde90  _warning
0003:000bde91  _error
0003:000bde92  _music_select
0003:000bde93  _killit_flag
0003:00006fb0  _spriteqamount
0003:00006fb4  _respawnactortime
0003:00006fb8  _respawnitemtime
0003:00006fbc  _weaponsandammosprites
0003:00006fdc  _dukefriction
0003:00006fe0  _freezerhurtowner
0003:00006fe1  _networkmode
0003:00006fe2  _movesperpacket
0003:00006fe3  _gamequit
0003:00006fe4  _numfreezebounces
0003:00006fe8  _bufferjitter
0003:00006fec  _cloudtotalclock
0003:00006ff0  _totalmemory
0003:00006ff4  _numinterpolations
0003:00006ff8  _startofdynamicinterpolations
0003:000bde94  _ready2send
0003:000bde95  _numplayersprites
0003:000bde96* _typebuflen
Module: menues.obj(H:\Games\duke3d\source\menues.c)
0003:000bdea0+ _minfo
0003:000bf058+ _numplr
0003:000bf05c+ _levnum
0003:000bf060+ _volnum
0003:000bf064+ _plrskl
0003:000bf068+ _mi
0003:000bf074* _deletespot
0003:000bf076+ _sh
0003:000bf078+ _last_zero
0003:000bf07a+ _onbar
0003:000bf07c+ _last_fifty
0003:000bf07e* _last_menu
0003:000bf080+ _buttonstat
0003:00006ffc  _probey
0003:00006ffe+ _lastprobey
0003:00007000  _globalskillsound
0003:00007002+ _last_threehundred
0001:00030570* dummyfunc_
0001:00030580* dummymess_
0001:00030590  cmenu_
0001:00030650  savetemp_
0001:00030680* getangplayers_
0001:000307a0+ loadpheader_
0001:00030900  loadplayer_
0001:00031730  saveplayer_
0001:00032140+ probe_
0001:00032540  menutext_
0001:00032860* menutextc_
0001:00032ab0+ bar_
0001:00032d50+ dispnames_
0001:00032f90+ getfilenames_
0001:000330a0+ sortfilenames_
0001:00033290  menus_
0001:00037660  palto_
0001:00037780  drawoverheadmap_
0001:00038830+ endanimsounds_
0001:00038990+ logoanimsounds_
0001:000389c0+ intro4animsounds_
0001:00038a00+ first4animsounds_
0001:00038a50* intro42animsounds_
0001:00038a60+ endanimvol41_
0001:00038a90+ endanimvol42_
0001:00038ad0+ endanimvol43_
0001:00038b10  playanm_
0003:00007006  _lastsavedpos
0003:00007008+ _quittimer
0003:0000700c+ _lastanimhack
Module: player.obj(H:\Games\duke3d\source\player.c)
0003:000bf090+ _dashow2dsector
0003:000bf190+ _searchparent
0003:000bfad0+ _searchsect
0003:000c0310  _lastvisinc
0003:000c0314+ _lastcontroltime
0003:000c0318+ _turnheldtime
0003:00007010  _myaimmode
0003:00007014+ _myaimstat
0003:00007018+ _omyaimstat
0003:0000701c+ _weapon_sprites
0001:00038f70  setpal_
0001:00039010+ incur_damage_
0001:00039120  quickkill_
0001:000391d0  forceplayerangle_
0001:00039210+ tracers_
0001:00039350  hits_
0001:00039440  hitasprite_
0001:000395a0  hitawall_
0001:00039640+ aim_
0001:00039b30  shoot_
0001:0003c3e0+ displayloogie_
0001:0003c510+ animatefist_
0001:0003c6b0+ animateknee_
0001:0003c830+ animateknuckles_
0001:0003c9a0  displaymasks_
0001:0003cb70+ animatetip_
0001:0003ccd0+ animateaccess_
0001:0003cfa0  displayweapon_
0001:0003ecc0  getinput_
0001:0003f5c0+ doincrements_
0001:0003fbd0  checkweapons_
0001:0003fca0  processinput_
0001:00043940+ getspritescore_
0001:00043d30  computergetinput_
0003:000c0324+ _fistsign
Module: premap.obj(H:\Games\duke3d\source\premap.c)
0001:00045bc0* tloadtile_
0001:00045be0+ cachespritenum_
0001:000460d0+ cachegoodsprites_
0001:000463c0+ getsound_
0001:000464c0+ precachenecessarysounds_
0001:00046500  cacheit_
0001:00046700  docacheit_
0001:000467a0  xyzmirror_
0001:00046880  vscrn_
0001:000469c0  pickrandomspot_
0001:00046a70+ resetplayerstats_
0001:00046d90  resetweapons_
0001:00046e30  resetinventory_
0001:00046ec0+ resetprestat_
0001:000470c0+ setupbackdrop_
0001:000471e0+ prelevel_
0001:00047d50  newgame_
0001:00047fa0+ resetpspritevars_
0001:000484c0+ clearfrags_
0001:00048540  resettimevars_
0001:00048580  genspriteremaps_
0001:000486b0  waitforeverybody_
0001:00048760+ dofrontscreens_
0001:00048950  clearfifo_
0001:00048b00  resetmys_
0001:00048bf0  enterlevel_
0003:00007274+ _which_palookup
Module: sector.obj(H:\Games\duke3d\source\sector.c)
0001:000490a0  callsound_
0001:000492b0  check_activator_motion_
0001:000493f0  isadoorwall_
0001:000494b0  isanunderoperator_
0001:00049530  isanearoperator_
0001:00049550  checkcursectnums_
0001:000495a0  ldist_
0001:000495d0  dist_
0001:00049600  findplayer_
0001:00049740  findotherplayer_
0001:00049810  doanimations_
0001:00049af0  getanimationgoal_
0001:00049b30+ setanimation_
0001:00049bd0  animatecamsprite_
0001:00049cb0  animatewalls_
0001:00049f70  activatewarpelevators_
0001:0004a150  operatesectors_
0001:0004b0b0  operaterespawns_
0001:0004b150  operateactivators_
0001:0004b450  operatemasterswitches_
0001:0004b4a0  operateforcefields_
0001:0004b580  checkhitswitch_
0001:0004c430  activatebysector_
0001:0004c4a0+ breakwall_
0001:0004c4e0  checkhitwall_
0001:0004ce30  checkplayerhurt_
0001:0004d0e0  checkhitceiling_
0001:0004d3c0  checkhitsprite_
0001:0004f100  allignwarpelevators_
0001:0004f250  cheatkeys_
0001:000500b0  checksectors_
0003:000c0348+ _haltsoundhack
Module: sounds.obj(H:\Games\duke3d\source\sounds.c)
0003:000c0350  _numenvsnds
0003:000c0354* _backflag
0001:00051120  SoundStartup_
0001:00051250  SoundShutdown_
0001:00051280  MusicStartup_
0001:00051360  MusicShutdown_
0001:000513a0  USRHOOKS_GetMem_
0001:000513c0  USRHOOKS_FreeMem_
0001:000513d0  intomenusounds_
0001:00051440  playmusic_
0001:000514c0+ loadsound_
0001:000515a0  xyzsound_
0001:00051cc0  sound_
0001:00051f00  spritesound_
0001:00051f50  stopsound_
0001:00051f90  stopenvsound_
0001:00052000  pan3dsound_
0001:00052390  testcallback_
0001:00052500  clearsoundlocks_
0003:00007278+ _menunum
Module: rts.obj(H:\Games\duke3d\source\rts.c)
0003:000c0368  _numlumps
0001:00052540+ RTS_AddFile_
0001:000526b0  RTS_Init_
0001:00052730  RTS_NumSounds_
0001:00052740+ RTS_SoundLength_
0001:00052780* RTS_GetSoundName_
0001:000527c0+ RTS_ReadLump_
0001:00052830  RTS_GetSound_
0003:000c0374  _lumplockbyte
Module: config.obj(H:\Games\duke3d\source\config.c)
0003:000c0384  _MusicToggle
0003:000c0388  _SoundToggle
0003:000c038c  _VoiceToggle
0003:000c0390  _AmbienceToggle
0003:000c0394  _ScreenHeight
0003:000c0398  _MixRate
0003:000c039c  _MouseAiming
0003:000c03a0  _ScreenMode
0003:000c03a4  _MidiPort
0003:000c03a8  _ControllerType
0003:000c03ac  _NumVoices
0003:000c03b0  _NumChannels
0003:000c03b4  _NumBits
0003:000c03b8  _ReverseStereo
0003:000c03bc  _ScreenWidth
0003:000c03c0  _BlasterConfig
0003:000c03dc  _FXVolume
0003:000c03e0  _MusicVolume
0003:000c03e4  _MusicDevice
0003:000c03e8  _FXDevice
0003:00007280+ _gamefunctions
0001:000528f0  CONFIG_GetSetupFilename_
0001:00052bf0+ CONFIG_FunctionNameToNum_
0001:00052c30* CONFIG_FunctionNumToName_
0001:00052c40+ CONFIG_AnalogNameToNum_
0001:00052cb0+ CONFIG_SetDefaults_
0001:00052d40+ CONFIG_ReadKeys_
0001:00052e30+ CONFIG_SetupMouse_
0001:00053070+ CONFIG_SetupGamePad_
0001:00053220+ CONFIG_SetupJoystick_
0001:00053480  readsavenames_
0001:00053540  CONFIG_ReadSetup_
0001:00053c50  CONFIG_WriteSetup_
Module: engine.obj(D:\engine.c)
0003:000c9124  _palookupoffse
0003:000c9134  _vince
0003:000c9144  _vplce
0003:000c9154  _bufplce
0003:000eb9f4+ _umost
0003:000ec674+ _dplc
0003:000edf74+ _uplc
0003:000f95f4+ _dmost
0003:000fa274+ _textfont
0003:000fa674+ _britable
0003:0010f8f4  _reciptable
0003:001118f4+ _smalltextfont
0003:00113774+ _tilefileoffs
0003:0011b774+ _slopalookup
0003:0011ea34+ _tilefilenum
0003:001214f4+ _picsiz
0003:00133cf4+ _voxlock
0003:001364f4+ _voxoff
0003:0013a1b4+ _visualpagelookup
0003:0013a2b4+ _activepagelookup
0003:0013a3b4+ _modelist
0003:0013a5b4  _show2dsector
0003:0013a634  _picanm
0003:00140634  _show2dwall
0003:00140a34  _tilesizx
0003:00143a34  _tilesizy
0003:00146a34+ _gotsector
0003:00146ab4  _walock
0003:001482b4  _gotpic
0003:001485b4  _nextspritestat
0003:0014a5b4  _waloff
0003:001505b4  _show2dsprite
0003:001507b4  _pskyoff
0003:001509b4+ _palookup
0003:00150db4  _sintable
0003:00151db4  _startumost
0003:00152a34  _prevspritesect
0003:00154a34  _startdmost
0003:001556b4  _nextspritesect
0003:001576b4  _prevspritestat
0003:001596b4  _palette
0003:001599b4  _sprite
0003:001859b4+ _validmode
0003:00185bb4  _wall
0003:001c5bb4  _tsprite
0003:001d0bb4+ _validmodexdim
0003:001d0fb4+ _validmodeydim
0003:001d13b4  _sector
0003:001db3d4+ _totalclocklock
0003:001db3e0+ _searchy
0003:001db450+ _ydim16
0003:001db454* _startposy
0003:001db458* _startposx
0003:001db45c* _startposz
0003:001db868+ _globalz
0003:001db86c+ _pageoffset
0003:001db870+ _globalx
0003:001db874+ _globaly
0003:001dba7c+ _globalx1
0003:001dba80  _globalx3
0003:001dba84+ _globalx2
0003:001dba88+ _globalorientation
0003:001dba8c+ _globalshade
0003:001dba90+ _globaly1
0003:001dba94  _globaly3
0003:001dba98+ _globaly2
0003:001dba9c+ _globalzd
0003:001dbaa0+ _globalzx
0003:001dbaa4+ _globalbufplc
0003:001dbaa8  _asm2
0003:001dbaac  _asm3
0003:001dbab0  _asm4
0003:001dbab4+ _globalyscale
0003:001dbab8+ _globalxpanning
0003:001dbabc+ _globalypanning
0003:001dbac0+ _xyaspect
0003:001dbac4+ _cosglobalang
0003:001dbac8+ _globaluclip
0003:001dbacc+ _globalcisibility
0003:001dbad0+ _sinviewingrangeglobalang
0003:001dbad4+ _globalposx
0003:001dbad8+ _globalhisibility
0003:001dbadc+ _globalposy
0003:001dbae0+ _globalposz
0003:001dbae4+ _globalvisibility
0003:001dbae8+ _cosviewingrangeglobalang
0003:001dbaec+ _globalpisibility
0003:001dbaf0+ _viewingrangerecip
0003:001dbaf4+ _globalpal
0003:001dbafc  _asm1
0003:001dbb00+ _globalhoriz
0003:001dbb04+ _globvis
0003:001dbb08+ _globalpalwritten
0003:001dbb0c+ _singlobalang
0003:001dbb10+ _globaldclip
0003:001dbb14+ _xdimenscale
0003:001dbb1c+ _xdimenrecip
0003:001dbb20+ _halfxdimen
0003:001dbb24+ _viewoffset
0003:001dbb28+ _wx2
0003:001dbb2c+ _wx1
0003:001dbb30+ _xdimscale
0003:001dbb34+ _wy2
0003:001dbb38+ _wy1
0003:001dbb3c+ _frameoffset
0003:001dbb44+ _ydimen
0003:001dcb4c+ _lastageclock
0003:001dcb50  _fpuasm
0003:001dcb54+ _activepage
0003:001dcb58+ _mapversion
0003:001dcb5c  _espbak
0003:001dcb60+ _artversion
0003:001dcb64+ _visualpage
0003:001dcb68+ _blackband
0003:001dcb6c+ _whiteband
0003:001dcb70  _ebpbak
0003:001dcf84+ _bytesperline
0003:001dcf88+ _origbuffermode
0003:001dcf8c+ _globlinplace
0003:001dcf94+ _xres
0003:001dcf98+ _imageSize
0003:001dcf9c+ _frameplace
0003:001dcfa0+ _maxpages
0003:001dcfa4+ _yres
0003:001dcfa8+ _linearmode
0003:001dcfac+ _buffermode
0003:001dcfb8+ _numtiles
0003:001dcfbc+ _VESABuf_rseg
0003:001dcfc0  _numframes
0003:001dcfc4+ _parallaxyoffs
0003:001dcfc8  _parallaxyscale
0003:001dcfcc  _windowy2
0003:001dcfd0  _windowy1
0003:001dcfd4  _randomseed
0003:001dcfd8  _windowx2
0003:001dcfdc  _windowx1
0003:001dcfe0+ _parallaxvisibility
0003:001dcfe4  _visibility
0003:001dcfe8  _ylookup
0003:001de2ac  _yxaspect
0003:001de2b0+ _validmodecnt
0003:001de2b4+ _numpages
0003:001de2b8  _spritesortcnt
0003:001de2bc  _totalclock
0003:001de2c0+ _viewingrange
0003:001de2c4  _ydim
0003:001de2c8  _xdim
0003:001de2cc+ _oldstereohandler
0003:001de2d2  _headspritestat
0003:001dead4  _headspritesect
0003:001df2d8+ _searchstat
0003:001df2da+ _searchsector
0003:001df2dc+ _searchwall
0003:001df2de+ _searchit
0003:001df2e2+ _numscans
0003:001df2e4+ _numbunches
0003:001df2e6+ _numhits
0003:001df2f0+ _highlightcnt
0003:001df2f2+ _linehighlight
0003:001df2f4* _startang
0003:001df2f6* _startsectnum
0003:001df2f8+ _pointhighlight
0003:001df2fa+ _globalpicnum
0003:001df2fc+ _globalshiftval
0003:001df2fe+ _globalang
0003:001df300+ _globalcursectnum
0003:001df306+ _oss
0003:001df308+ _ods
0003:001df30a+ _oes
0003:001df30c  _pskybits
0003:001df30e+ _numpalookups
0003:001df310  _numwalls
0003:001df312  _numsectors
0003:001df391+ _globalxshift
0003:001df392+ _globalyshift
0003:001df393+ _globparaceilclip
0003:001df394+ _globparaflorclip
0003:001df395+ _o3c2
0003:001df396+ _ortca
0003:001df397+ _ortcb
0003:000073d4+ _VESABuf_len
0003:000073d8+ _VESABuf_sel
0003:000073e1+ _setactiveentry
0003:000073e5+ _setvisualentry
0003:000073e9+ _setpaletteentry
0003:000073ed+ _permanentupdate
0003:000073f3+ _transarea
0003:000073f7+ _totalarea
0003:000073fb+ _beforedrawrooms
0003:0000740b+ _stereowidth
0003:0000740f+ _stereopixelwidth
0003:00007413+ _ostereopixelwidth
0003:00007417+ _stereomode
0003:00007420+ _pic
0003:00007424+ _artsize
0003:00007428+ _cachesize
0003:0000742c  _pow2char
0003:00007434  _pow2long
0003:000074b8+ _xdimen
0003:000074bd+ _qsetmode
0003:000074c1+ _transluc
0003:000074c5+ _paletteloaded
0003:000074ce+ _hitscangoalx
0003:000074d2+ _hitscangoaly
0003:00007590+ _editstatus
0003:00007592+ _searchx
0003:0000759b  _cachedebug
0003:0000759c+ _clipmoveboxtracenum
0001:00053f97+ DPMI_int86_
0001:000540aa+ DPMI_int86x_
0001:00054249+ VBE_callESDI_
0001:00054349* VBE_getModeInfo_
0001:00054387+ GetPtrToLFB_
0001:000545d3+ getvalidvesamodes_
0001:00054878+ setvesa_
0001:00054bf5* setdacbits_
0001:00054c35+ setactivepage_
0001:00054cdc+ setvisualpage_
0001:0005544b+ uninitvesa_
0001:0005546b  VBE_setPalette_
0001:00055581+ VBE_getPalette_
0001:0005560b+ loadvoxel_
0001:0005560c  kmalloc_
0001:00055611  kfree_
0001:00055616  drawrooms_
0001:00055cbf+ scansector_
0001:0005641b+ wallfront_
0001:00056641+ spritewallfront_
0001:00056695+ bunchfront_
0001:0005672f+ drawalls_
0001:0005793c+ prepwall_
0001:00057cb2+ ceilscan_
0001:000585e5+ florscan_
0001:00058f6a+ wallscan_
0001:00059a5b+ maskwallscan_
0001:0005a561+ transmaskwallscan_
0001:0005a63a  loadboard_
0001:0005a7ee* saveboard_
0001:0005a969+ loadtables_
0001:0005aa4d+ loadpalette_
0001:0005ac91  setgamemode_
0001:0005af5c+ hline_
0001:0005b01b+ slowhline_
0001:0005b14d+ transmaskvline_
0001:0005b2bf+ transmaskvline2_
0001:0005b6dd  initengine_
0001:0005b830  uninitengine_
0001:0005b8d9  nextpage_
0001:0005bbe6  loadtile_
0001:0005bd5e* allocatepermanenttile_
0001:0005be17  loadpics_
0001:0005c11a* qloadkvx_
0001:0005c1ca  clipinsidebox_
0001:0005c2b5+ clipinsideboxline_
0001:0005c396+ readpixel16_
0001:0005c46b  screencapture_
0001:0005c972  inside_
0001:0005ca21  getangle_
0001:0005cb06  ksqrt_
0001:0005cb3a* krecip_
0001:0005cb76+ initksqrt_
0001:0005cc24* copytilepiece_
0001:0005cd6a  drawmasks_
0001:0005d3dd+ drawmaskwall_
0001:0005d912+ drawsprite_
0001:00060b77+ drawvox_
0001:00061966+ ceilspritescan_
0001:00061a3e+ ceilspritehline_
0001:00061baf  setsprite_
0001:00061c11+ animateoffs_
0001:00061c9c+ initspritelists_
0001:00061d71  insertsprite_
0001:00061d86+ insertspritesect_
0001:00061e22+ insertspritestat_
0001:00061ebe  deletesprite_
0001:00061ed2+ deletespritesect_
0001:00061faa+ deletespritestat_
0001:00062080  changespritesect_
0001:000620c7  changespritestat_
0001:0006210e  nextsectorneighborz_
0001:000621d6  cansee_
0001:0006244a  hitscan_
0001:000635c5  neartag_
0001:00063bde+ lintersect_
0001:00063d01+ rintersect_
0001:00063e01  dragpoint_
0001:00063eae+ lastwall_
0001:00063efe  clipmove_
0001:000656cc+ keepaway_
0001:0006576f+ raytrace_
0001:0006596d  pushmove_
0001:00065d20  updatesector_
0001:00065dd8  rotatepoint_
0001:00065e70* initmouse_
0001:00065e86* getmousevalues_
0001:00065eca* printscreeninterrupt_
0001:00065ecd  drawline256_
0001:0006622c+ drawline16_
0001:000666f2* qsetmode640350_
0001:00066775* qsetmode640480_
0001:00066868+ clear2dscreen_
0001:000668ca+ draw2dgrid_
0001:00066b75* draw2dscreen_
0001:0006777b* printext16_
0001:00067a2e  printext256_
0001:00067b28  krand_
0001:00067b3c  getzrange_
0001:0006864c  setview_
0001:00068813  setaspect_
0001:00068878+ dosetaspect_
0001:00068a16  flushperms_
0001:00068a27  rotatesprite_
0001:00068dd1+ dorotatesprite_
0001:0006a998+ clippoly4_
0001:0006ac35  makepalookup_
0001:0006aedb+ initfastcolorlookup_
0001:0006b0c5+ getclosestcol_
0001:0006b2a3  setbrightness_
0001:0006b3a5  drawmapview_
0001:0006c873+ clippoly_
0001:0006d6ba+ fillpolygon_
0001:0006db1e  clearview_
0001:0006dca1+ clearallviews_
0001:0006dd86* plotpixel_
0001:0006dda8* getpixel_
0001:0006ddc2  setviewtotile_
0001:0006df6e  setviewback_
0001:0006e0e5  squarerotatetile_
0001:0006e199  preparemirror_
0001:0006e3aa  completemirror_
0001:0006e5a0* sectorofwall_
0001:0006e64a  getceilzofslope_
0001:0006e728  getflorzofslope_
0001:0006e806  getzsofslope_
0001:0006e92a* alignceilslope_
0001:0006e9f8  alignflorslope_
0001:0006eac7+ owallmost_
0001:0006ef7e+ wallmost_
0001:0006f8f5+ grouscan_
0001:00070551+ getpalookup_
0001:0007057f+ parascan_
0001:00070bba+ stereohandler_
0001:00070c58+ initstereo_
0001:00070e1c+ uninitstereo_
0001:00070f4d+ stereonextpage_
0001:000710a2+ loopnumofsector_
0001:000710f5* setfirstwall_
0003:001df399+ _oa1
0003:001df39a+ _overtbits
0003:001df39b+ _laststereoint
0003:001df39c  _vgacompatible
0003:001df39d  _automapping
0003:001df39e  _parallaxtype
0003:001df39f+ _showinvisibility
0003:001df3a0+ _vidoption
Module: cache1d.obj(C:\C\CPROG\BUILD\cache1d.c)
0003:001df524  _cac
0003:000075a8+ _cachecount
0003:000075ac+ _zerochar
0003:000075ad+ _cachestart
0003:000075b1  _cacnum
0003:000075b5+ _agecount
0001:00071372  initcache_
0001:000713d1  allocache_
0001:00071705  suckcache_
0001:00071848  agecache_
0001:000718c1+ reportandexit_
0001:00071985  initgroupfile_
0001:00071b69  uninitgroupfile_
0001:00071bb7  kopen4load_
0001:00071ce9  kread_
0001:00071dee  klseek_
0001:00071e6d  kfilelength_
0001:00071eae  kclose_
0001:00071ed9  kdfread_
0001:000720f6  dfread_
0001:00072303  dfwrite_
0001:0007257f+ compress_
0001:00072798+ uncompress_
Module: mmulti.obj(C:\C\CPROG\2DRAW\mmulti.c)
0003:001f9878+ _crctable
0003:001f9f18  _connectpoint2
0003:001fa020  _connecthead
0003:001fa024  _numplayers
0003:001fa026  _myconnectindex
0001:00072904+ callcommit_
0001:00072932  initmultiplayers_
0001:00072a60+ initcrc_
0001:00072ab9  setpackettimeout_
0001:00072ae4+ getcrc_
0001:00072b2b  sendlogon_
0001:00072b2b  uninitmultiplayers_
0001:00072b2c  sendlogoff_
0001:00072b74  getoutputcirclesize_
0001:00072b76* setsocket_
0001:00072b77  sendpacket_
0001:00072c77+ dosendpackets_
0001:00072ec3  getpacket_
0001:000731b5  flushpackets_
0001:000731b6  genericmultifunction_
0003:000077dd  _syncstate
Module: a.obj(a.asm)
0001:000a4210  qrhlineasm4_
0001:000a2e50  setvlinebpl_
0001:000a382c  spritevline_
0001:000a3850  msetupspritevline_
0001:000a38c0  tsetupspritevline_
0001:000a3190  prevlineasm1_
0001:000a3980  mhline_
0001:000a3af0  thline_
0001:000a44b9* STRETCHHLINE_
0001:000a2ea0  setpalookupaddress_
0001:000a38a0  mspritevline_
0001:000a38f0  tspritevline_
0001:000a42af  setupdrawslab_
0001:000a2da0  sethlinesizes_
0001:000a3100  setupvlineasm_
0001:000a4310  drawslab_
0001:000a2ed0  setuphlineasm4_
0001:000a3950  msethlineshift_
0001:000a3ac0  tsethlineshift_
0001:000a3240  settransnormal_
0001:000a3160  setupmvlineasm_
0001:000a3180  setuptvlineasm_
0001:000a2f10  hlineasm4_
0001:000a3e20  setupslopevlin_
0001:000a31b0  vlineasm1_
0001:000a3380  vlineasm4_
0001:000a3f80  setuprhlineasm4_
0001:000a3c20  setuptvlineasm2_
0001:000a3e70  slopevlin_
0001:000a3d70* SETUPSLOPEVLIN2_
0001:000a32c0  settransreverse_
0001:000a4020  rhlineasm4_
0001:000a31e0  mvlineasm1_
0001:000a3560  mvlineasm4_
0001:000a3340  tvlineasm1_
0001:000a3c50  tvlineasm2_
0001:000a3dc0* SLOPEVLIN2_
0001:000a4130  setuprmhlineasm4_
0001:000a41b0  setupqrhlineasm4_
0001:000a39d0* MHLINESKIPMODIFY_
0001:000a3210  fixtransluscence_
0001:000a3b40* THLINESKIPMODIFY_
0001:000a37e0  setupspritevline_
0001:000a4150  rmhlineasm4_
Module: animlib.obj(H:\Games\duke3d\source\animlib.c)
0003:000077e0  _anim
0001:00073210+ CheckAnimStarted_
0001:00073230+ findpage_
0001:00073290+ loadpage_
0001:00073330+ CPlayRunSkipDump_
0001:000733b0+ renderframe_
0001:00073450+ drawframe_
0001:000734a0  ANIM_LoadAnim_
0001:00073570  ANIM_FreeAnim_
0001:00073590  ANIM_NumFrames_
0001:000735b0  ANIM_DrawFrame_
0001:00073630  ANIM_GetPalette_
Module: audio_wf.lib(D:\PRG\AUDIO\source\task_man.c)
0001:00073864  TS_Shutdown_
0001:000738d4  TS_ScheduleTask_
0001:000739dc  TS_Terminate_
0001:00073a4c  TS_Dispatch_
0001:00073a88  TS_SetTaskRate_
0001:00073ac4+ TS_UnlockMemory_
0001:00073b24+ TS_LockMemory_
0003:000077f8+ _TS_InInterrupt
Module: H:\WATCOM\lib386\dos\clib3r.lib(toupper)
0001:00073ba0  toupper_
Module: H:\WATCOM\lib386\dos\clib3r.lib(ltoa)
0001:00073bb0  ultoa_
0001:00073c00  ltoa_
Module: mact\mact386.lib(P:\LIBMACT\keyboard.c)
0003:001fa160  _KB_KeyDown
0001:00073c30  KB_KeyEvent_
0001:00073cec  KB_KeyWaiting_
0001:00073d00  KB_Getch_
0001:00073d40* KB_Addch_
0001:00073d6c* KB_TurnKeypadOn_
0001:00073d78* KB_TurnKeypadOff_
0001:00073d84* KB_KeypadActive_
0001:00073d8c  KB_FlushKeyBoardQueue_
0001:00073da0  KB_ClearKeysDown_
0001:00073dc0* KB_ScanCodeToString_
0001:00073dd4  KB_StringToScanCode_
0001:00073e04  KB_Startup_
0001:00073e58  KB_Shutdown_
0003:001fa1ec+ _KB_LastScan
Module: audio_wf.lib(D:\PRG\AUDIO\source\fx_man.c)
0001:00073ef4  FX_ErrorString_
0001:00073ff4* FX_SetupCard_
0001:00074198* FX_GetBlasterSettings_
0001:00074200  FX_SetupSoundBlaster_
0001:000742d0  FX_Init_
0001:000743c8  FX_Shutdown_
0001:00074460  FX_SetCallBack_
0001:000744c8  FX_SetVolume_
0001:00074548* FX_GetVolume_
0001:00074584  FX_SetReverseStereo_
0001:0007458c  FX_GetReverseStereo_
0001:00074594  FX_SetReverb_
0001:0007459c* FX_SetFastReverb_
0001:000745a4* FX_GetMaxReverbDelay_
0001:000745ac* FX_GetReverbDelay_
0001:000745b4  FX_SetReverbDelay_
0001:000745bc  FX_VoiceAvailable_
0001:000745c4* FX_SetPan_
0001:000745e4* FX_SetPitch_
0001:00074604* FX_SetFrequency_
0001:00074624* FX_PlayVOC_
0001:00074658  FX_PlayLoopedVOC_
0001:00074698* FX_PlayWAV_
0001:000746cc  FX_PlayLoopedWAV_
0001:0007470c  FX_PlayVOC3D_
0001:0007473c  FX_PlayWAV3D_
0001:0007476c* FX_PlayRaw_
0001:000747ac* FX_PlayLoopedRaw_
0001:000747f8  FX_Pan3D_
0001:00074818* FX_SoundActive_
0001:00074820* FX_SoundsPlaying_
0001:00074828  FX_StopSound_
0001:00074844  FX_StopAllSounds_
0001:00074860* FX_StartDemandFeedPlayback_
0001:0007489c* FX_StartRecording_
0001:000748e0* FX_StopRecord_
0003:00007ab4+ _FX_SoundDevice
0003:00007ab8+ _FX_ErrorCode
0003:00007abc+ _FX_Installed
Module: H:\WATCOM\lib386\dos\clib3r.lib(printf)
0001:00074900  printf_
Module: H:\WATCOM\lib386\dos\clib3r.lib(sprintf)
0001:00074930  sprintf_
Module: H:\WATCOM\lib386\dos\clib3r.lib(unlnk)
0001:00074960  unlink_
Module: H:\WATCOM\lib386\dos\clib3r.lib(exit)
0001:00074990  __null_int23_exit_
0001:000749b0  exit_
0001:000749e0+ _exit_
0003:00007ac0  ___int23_exit
0003:00007ac4  ___FPE_handler_exit
Module: H:\WATCOM\lib386\dos\clib3r.lib(fclose)
0001:00074a00  fclose_
0001:00074a30  __shutdown_stream_
0001:00074a50  __doclose_
0003:001fa200+ ___RmTmpFileFn
Module: mact\mact386.lib(P:\LIBMACT\mathutil.c)
0001:00074ae0  FindDistance2D_
0001:00074b3c  FindDistance3D_
0001:00074b94* FindDistance3D_HP_
0001:00074c38* ArcTangentAppx_
Module: H:\WATCOM\lib386\dos\clib3r.lib(rand)
0001:00074d00  rand_
0001:00074d30* srand_
Module: H:\WATCOM\lib386\dos\clib3r.lib(tolower)
0001:00074d50  tolower_
Module: mact\mact386.lib(P:\LIBMACT\control.c)
0003:001fa820+ _CONTROL_JoysPresent
0003:00007acc  _CONTROL_RudderEnabled
0003:00007ad0+ _CONTROL_MouseEnabled
0003:00007ad4+ _CONTROL_ExternalEnabled
0003:00007ad8  _CONTROL_JoystickEnabled
0003:00007adc  _CONTROL_JoystickPort
0001:00074d60+ CONTROL_GetMouseDelta_
0001:00074dd0  CONTROL_GetMouseSensitivity_
0001:00074ddc  CONTROL_SetMouseSensitivity_
0001:00074de8* CONTROL_GetMouseButtons_
0001:00074df0* CONTROL_StartMouse_
0001:00074e00+ CONTROL_GetJoyAbs_
0001:00074e8c+ CONTROL_FilterJoyDelta_
0001:00074f3c+ CONTROL_GetJoyDelta_
0001:00074fa8+ CONTROL_JoyButtons_
0001:00075058+ CONTROL_SetJoyScale_
0001:000750e8+ CONTROL_SetupJoy_
0001:00075170  CONTROL_CenterJoystick_
0001:000753d0+ CONTROL_StartJoy_
0001:00075438* CONTROL_ShutJoy_
0001:00075444+ CONTROL_ExternalStartup_
0001:000754d4+ CONTROL_ExternalSetup_
0001:000755a4+ CONTROL_PollExternalControl_
0001:00075614+ CONTROL_GetTime_
0001:00075628+ CONTROL_CheckRange_
0001:00075644+ CONTROL_SetFlag_
0001:0007569c+ CONTROL_KeyboardFunctionPressed_
0001:000756f0* CONTROL_ClearKeyboardFunction_
0001:00075728  CONTROL_DefineFlag_
0001:00075784* CONTROL_FlagActive_
0001:0007579c  CONTROL_MapKey_
0001:000757b4* CONTROL_PrintKeyMap_
0001:000757e8* CONTROL_PrintControlFlag_
0001:00075830* CONTROL_PrintAxes_
0001:00075880  CONTROL_MapButton_
0001:000758c4  CONTROL_MapAnalogAxis_
0001:00075904  CONTROL_SetAnalogAxisScale_
0001:0007592c  CONTROL_MapDigitalAxis_
0001:00075978* CONTROL_ClearFlags_
0001:00075990  CONTROL_ClearAssignments_
0001:00075a08+ CONTROL_GetDeviceButtons_
0001:00075b20+ CONTROL_DigitizeAxis_
0001:00075b94* CONTROL_ScaleAxis_
0001:00075bd8+ CONTROL_ApplyAxis_
0001:00075c3c+ CONTROL_PollDevices_
0001:00075da0+ CONTROL_AxisFunctionState_
0001:00075e00+ CONTROL_ButtonFunctionState_
0001:00075e58+ CONTROL_GetUserInput_
0001:00075ff0+ CONTROL_ClearUserInput_
0001:00076168  CONTROL_ClearButton_
0001:000761c4  CONTROL_GetInput_
0001:000762bc* CONTROL_WaitRelease_
0001:000762e0* CONTROL_Ack_
0001:00076380  CONTROL_Startup_
0001:000765f0  CONTROL_Shutdown_
0003:001fa848+ _CONTROL_ButtonHeldState1
0003:001fa84c+ _CONTROL_ButtonHeldState2
0003:001fa850  _CONTROL_MousePresent
0003:001fa854  _CONTROL_ButtonState1
0003:001fa858  _CONTROL_ButtonState2
Module: H:\WATCOM\lib386\dos\clib3r.lib(puts)
0001:00076620  puts_
Module: mact\mact386.lib(P:\LIBMACT\file_lib.c)
0001:00076650+ SafeOpen_
0001:000766f0  SafeOpenWrite_
0001:00076730  SafeOpenRead_
0001:0007676c* SafeOpenAppend_
0001:000767ac  SafeClose_
0001:0007680c  SafeFileExists_
0001:00076820* SafeFileLength_
0001:00076828  SafeRead_
0001:00076898  SafeWrite_
0001:00076908  LoadFile_
0001:0007693c* SaveFile_
0001:0007695c* GetPathFromEnvironment_
0001:00076a18* DefaultExtension_
0001:00076a74* DefaultPath_
0001:00076af0* ExtractFileBase_
0001:00076b60* GetExtension_
0001:00076bb8* SetExtension_
0001:00076c0c+ GetPath_
0001:00076c58* ChangeDirectory_
0001:00076cdc+ ChangeDrive_
Module: H:\WATCOM\lib386\dos\clib3r.lib(atol)
0001:00076d20  atol_
Module: audio_wf.lib(D:\PRG\AUDIO\source\music.c)
0003:00007b60  _MUSIC_SoundDevice
0003:00007b64  _MUSIC_ErrorCode
0001:00076dbd  MUSIC_ErrorString_
0001:00076e5f  MUSIC_Init_
0001:00076f55  MUSIC_Shutdown_
0001:00076fd1* MUSIC_SetMaxFMMidiChannel_
0001:00076fd6  Music_SetVolume_
0001:00076ff6* MUSIC_SetMidiChannelVolume_
0001:00076ffb* MUSIC_ResetMidiChannelVolumes_
0001:00077000* MUSIC_GetVolume_
0001:00077010* MUSIC_SetLoopFlag_
0001:00077015* MUSIC_SongPlaying_
0001:0007701a  MUSIC_Continue_
0001:0007701f  MUSIC_Pause_
0001:00077024  MUSIC_StopSong_
0001:00077053  MUSIC_PlaySong_
0001:00077094* MUSIC_SetContext_
0001:00077099* MUSIC_GetContext_
0001:0007709e* MUSIC_SetSongTick_
0001:000770a3* MUSIC_SetSongTime_
0001:000770a8* MUSIC_SetSongPosition_
0001:000770ad* MUSIC_GetSongPosition_
0001:000770b2* MUSIC_GetSongLength_
0001:000770b7+ MUSIC_InitAWE32_
0001:00077138+ MUSIC_InitFM_
0001:000771f1+ MUSIC_InitMidi_
0001:000772b5+ MUSIC_InitGUS_
0001:0007737f* MUSIC_FadeVolume_
0001:0007746b* MUSIC_FadeActive_
0001:0007747b* MUSIC_StopFade_
0001:00077499* MUSIC_RerouteMidiChannel_
0001:0007749e  MUSIC_RegisterTimbreBank_
Module: H:\WATCOM\lib386\dos\clib3r.lib(fopen)
0001:000774b0+ __open_flags_
0001:000776e0+ _fsopen_
0001:00077730  fopen_
0001:000777b0* freopen_
Module: H:\WATCOM\lib386\dos\clib3r.lib(fprintf)
0001:00077810  fprintf_
Module: H:\WATCOM\lib386\dos\clib3r.lib(int386)
0001:00077840  int386_
Module: H:\WATCOM\lib386\dos\clib3r.lib(intx386)
0001:00077860  int386x_
Module: H:\WATCOM\lib386\dos\clib3r.lib(open)
0001:00077880  open_
0001:000778a0  sopen_
0001:00077b30* __set_binary_
Module: H:\WATCOM\lib386\dos\clib3r.lib(filelen)
0001:00077ba0  filelength_
Module: H:\WATCOM\lib386\dos\clib3r.lib(close)
0001:00077bf0  close_
Module: mact\mact386.lib(P:\LIBMACT\zone.c)
0001:00077d50+ Z_FreeZone_
0001:00077d98* Z_Init_
0001:00077db8* Z_ShutDownZone_
0001:00077dd4* Z_ShutDown_
0001:00077df8* Z_GetSize_
0001:00077e28+ Z_AddFreeBlock_
0001:00077ea4+ Z_FreeBlock_
0001:00077ef8+ Z_Free_
0001:00077f2c* Z_FreeTags_
0001:00077f88+ Z_PurgeZone_
0001:00077fe4* Z_FindBlockInFreeList_
0001:00078010+ Z_FindFreeBlock_
0001:00078074+ Z_Malloc_
0001:00078174* Z_Touch_
0001:000781d8* Z_Realloc_
0001:00078250* Z_ZoneUsed_
0001:00078294* Z_ZoneMaxFree_
0001:000782d8* Z_ZoneSize_
0001:000782fc* Z_ChangeTag_
0001:0007832c  Z_AvailHeap_
0001:00078380* Z_DumpHeap_
0001:00078494* Z_CheckHeap_
Module: mact\mact386.lib(P:\LIBMACT\util_lib.c)
0001:00078544  RegisterShutdownFunction_
0001:0007854c  Error_
0001:000785b0  CheckParm_
0001:0007863c+ ParseHex_
0001:000786cc* ParseNum_
0001:000786f8* MotoShort_
0001:00078710* IntelShort_
0001:00078714* MotoLong_
0001:00078760  IntelLong_
0001:00078764* HeapSort_
0001:00078894  SafeMalloc_
0001:000788b8* SafeMallocSize_
0001:000788c0  SafeRealloc_
0001:000788e4  SafeFree_
Module: H:\WATCOM\lib386\dos\clib3r.lib(fwrite)
0001:00078910  fwrite_
Module: H:\WATCOM\lib386\dos\clib3r.lib(fseek)
0001:00078b80  fseek_
Module: H:\WATCOM\lib386\dos\clib3r.lib(cstart)
0001:00000003* ___begtext
0003:00000000* __nullarea
0003:00007b94  __GDAptr
0003:00007b98  __D16Infoseg
0003:00007b9a  __x386_zero_base_selector
0001:00078c94  _cstart_
0001:00078f0b  __exit_
0001:00078f0d  __do_exit_with_msg__
0001:00078f48  __GETDS
0001:00078f48  ___GETDSStart_
0001:00078f53  ___GETDSEnd_
Module: H:\WATCOM\lib386\dos\clib3r.lib(argcv)
0003:001fa8ec  __argc
0003:001fa8f0  __argv
0003:001fa8f4  ___argc
0003:001fa8f8  ___argv
Module: H:\WATCOM\lib386\dos\clib3r.lib(istable)
0003:000067c8  __IsTable
Module: H:\WATCOM\lib386\dos\clib3r.lib(_strcmp)
0001:00078f60  strcmp_
Module: H:\WATCOM\lib386\dos\clib3r.lib(write)
0001:000791b0  write_
Module: H:\WATCOM\lib386\dos\clib3r.lib(dosfind)
0001:000793fe  _dos_findfirst_
0001:0007941b  _dos_findnext_
0001:00079437* _dos_findclose_
Module: mact\mact386.lib(P:\LIBMACT\vidmsdos.c)
0003:0020a300+ _vid_flushall
0001:00079480* VID_Init_
0001:00079528* VID_Shutdown_
0001:0007954c* VID_GetBuffer_
0001:00079550* VID_Update_
0001:00079574* VID_UpdateScreen_
0001:0007959c* VID_NormalizePalette_
0001:000795bc* VID_GetPalette_
0001:000795ec* VID_SetPalette_
0001:0007961c* VID_ClearViewBuffer_
0001:00079638  ServiceEvents_
0001:0007963c* MOUSE_ShowCursor_
0001:00079664* MOUSE_HideCursor_
0001:0007968c* MOUSE_GetPosition_
0001:000796c8  MOUSE_GetDelta_
0001:00079704  MOUSE_GetButtons_
0001:00079730  MOUSE_Init_
0001:00079760  MOUSE_Shutdown_
0001:00079864  KEYBOARD_Startup_
0001:000798b4  KEYBOARD_Shutdown_
0003:0020a30c+ _vid
Module: H:\WATCOM\lib386\dos\clib3r.lib(nmalloc)
0001:00079910  malloc_
0001:00079920  _nmalloc_
0003:00007c30  ___nheapbeg
0003:00007c34  ___MiniHeapRover
0003:00007c38  ___LargestSizeB4MiniHeapRover
Module: H:\WATCOM\lib386\dos\clib3r.lib(nfree)
0001:00079a30  free_
0001:00079a40  _nfree_
0003:0020a330  ___MiniHeapFreeRover
Module: H:\WATCOM\lib386\dos\clib3r.lib(strncmp)
0001:00079b50  strncmp_
Module: H:\WATCOM\lib386\dos\clib3r.lib(stack386)
0001:00079b80  stackavail_
Module: H:\WATCOM\lib386\dos\clib3r.lib(stk)
0001:00079ba5* __STK
0001:00079b92  __CHK
0001:00079ba2  __GRO
0001:00079bc3  __STKOVERFLOW_
Module: H:\WATCOM\lib386\dos\clib3r.lib(lseek)
0001:00079be0  lseek_
Module: H:\WATCOM\lib386\dos\clib3r.lib(strncpy)
0001:00079c50  strncpy_
Module: H:\WATCOM\lib386\dos\clib3r.lib(memset)
0001:00079c90  memset_
Module: H:\WATCOM\lib386\dos\clib3r.lib(clock)
0001:00079cd0  clock_
Module: H:\WATCOM\lib386\dos\clib3r.lib(_istrcmp)
0001:00079d52  strcmpi_
Module: H:\WATCOM\lib386\dos\clib3r.lib(iob)
0003:00007c50  ___iob
0003:00007e58  __fmode
0003:0020a348  ___OpenStreams
0003:0020a34c  ___ClosedStreams
Module: H:\WATCOM\lib386\dos\clib3r.lib(fflush)
0001:00079d60  fflush_
Module: H:\WATCOM\lib386\dos\clib3r.lib(stricmp)
0001:00079d70  stricmp_
Module: mact\mact386.lib(P:\LIBMACT\scriplib.c)
0001:00079db0* SCRIPT_HandleValid_
0001:00079dc4+ SCRIPT_New_
0001:00079e34+ SCRIPT_Delete_
0001:00079e70+ SCRIPT_Init_
0001:00079f10+ SCRIPT_FreeSection_
0001:00079f74  SCRIPT_Free_
0001:0007a050+ SCRIPT_Parse_
0001:0007a0ac  SCRIPT_Load_
0001:0007a0ec* SafeWriteString_
0001:0007a10c  SCRIPT_Save_
0001:0007a208* SCRIPT_AddLine_
0001:0007a22c+ SCRIPT_SectionExists_
0001:0007a288+ SCRIPT_AddSection_
0001:0007a288* SCRIPT_PutSection_
0001:0007a3a0* SCRIPT_EntryExists_
0001:0007a3d4+ SCRIPT_AddEntry_
0001:0007a3d4* SCRIPT_PutRaw_
0001:0007a570+ SCRIPT_DecodeToken_
0001:0007a714+ SCRIPT_NumberSections_
0001:0007a760* SCRIPT_Section_
0001:0007a7d8  SCRIPT_NumberEntries_
0001:0007a824  SCRIPT_Entry_
0001:0007a898+ SCRIPT_GetRaw_
0001:0007a900  SCRIPT_GetString_
0001:0007a998  SCRIPT_GetDoubleString_
0001:0007aab8  SCRIPT_GetNumber_
0001:0007ab20* SCRIPT_GetBoolean_
0001:0007ab7c* SCRIPT_GetDouble_
0001:0007abc0+ SCRIPT_PutComment_
0001:0007ac6c* SCRIPT_PutEOL_
0001:0007ac7c* SCRIPT_PutMultiComment_
0001:0007acd0  SCRIPT_PutString_
0001:0007acfc* SCRIPT_PutDoubleString_
0001:0007ad34  SCRIPT_PutNumber_
0001:0007ad90* SCRIPT_PutBoolean_
0001:0007adc4* SCRIPT_PutDouble_
Module: H:\WATCOM\lib386\dos\clib3r.lib(segread)
0001:0007ae20  segread_
Module: H:\WATCOM\lib386\dos\clib3r.lib(atexit)
0001:0007ae50  atexit_
Module: H:\WATCOM\lib386\dos\clib3r.lib(fmemcpy)
0001:0007aec0  _fmemcpy_
Module: H:\WATCOM\lib386\dos\clib3r.lib(ldiv386)
0001:0007aee8  div_
0001:0007aee8* ldiv_
Module: H:\WATCOM\lib386\dos\clib3r.lib(strlen)
0001:0007af00  strlen_
Module: H:\WATCOM\lib386\dos\clib3r.lib(strcpy)
0001:0007af20  strcpy_
Module: H:\WATCOM\lib386\dos\clib3r.lib(disable)
0001:0007af40  _disable_
Module: H:\WATCOM\lib386\dos\clib3r.lib(d_getvec)
0001:0007af50  _dos_getvect_
Module: H:\WATCOM\lib386\dos\clib3r.lib(d_setvec)
0001:0007af90  _dos_setvect_
Module: H:\WATCOM\lib386\dos\clib3r.lib(enable)
0001:0007afc0  _enable_
Module: H:\WATCOM\lib386\dos\clib3r.lib(memcpy)
0001:0007afd0  memcpy_
Module: H:\WATCOM\lib386\dos\clib3r.lib(read)
0001:0007b000  read_
Module: H:\WATCOM\lib386\dos\clib3r.lib(min)
0001:0007b150  min_
Module: H:\WATCOM\lib386\dos\clib3r.lib(fread)
0001:0007b160  fread_
Module: H:\WATCOM\lib386\dos\clib3r.lib(strtok)
0001:0007b380  strtok_
Module: H:\WATCOM\lib386\dos\clib3r.lib(chainint)
0001:0007b41c  _chain_intr_
Module: audio_wf.lib(D:\PRG\AUDIO\source\dpmi.c)
0001:0007b440* DPMI_GetRealModeVector_
0001:0007b484* DPMI_SetRealModeVector_
0001:0007b4c0  DPMI_CallRealModeFunction_
0001:0007b524  DPMI_LockMemoryRegion_
0001:0007b528  DPMI_LockMemory_
0001:0007b580  DPMI_UnlockMemoryRegion_
0001:0007b584  DPMI_UnlockMemory_
Module: audio_wf.lib(D:\PRG\AUDIO\source\blaster.c)
0003:0020a468+ _BLASTER_Version
0003:0020a470+ _BLASTER_SoundPlaying
0003:0020a474+ _BLASTER_CallBack
0003:0020a47c+ _BLASTER_SoundRecording
0003:0020a494+ _BLASTER_Card
0003:0020a4a8  _BLASTER_DMAChannel
0003:00007e64  _BLASTER_Config
0001:0007b5e0+ _BLASTER_Interrupts
0001:0007b620+ _BLASTER_SampleSize
0001:0007b630* _BLASTER_CardConfig
0001:0007b6fc  BLASTER_ErrorString_
0001:0007b780+ BLASTER_EnableInterrupt_
0001:0007b7d0+ BLASTER_DisableInterrupt_
0001:0007b848+ BLASTER_ServiceInterrupt_
0001:0007b9a0+ BLASTER_ReadDSP_
0001:0007b9ec+ BLASTER_ResetDSP_
0001:0007ba4c+ BLASTER_GetDSPVersion_
0001:0007bb60* BLASTER_SpeakerOn_
0001:0007bb68* BLASTER_SpeakerOff_
0001:0007bb70+ BLASTER_WriteDSP_
0001:0007bba8+ BLASTER_SetPlaybackRate_
0001:0007bccc  BLASTER_GetPlaybackRate_
0001:0007bcd4  BLASTER_SetMixMode_
0001:0007bd54  BLASTER_StopPlayback_
0001:0007bdb4+ BLASTER_SetupDMABuffer_
0001:0007be38  BLASTER_GetCurrentPos_
0001:0007beac+ BLASTER_DSP1xx_BeginPlayback_
0001:0007beec+ BLASTER_DSP2xx_BeginPlayback_
0001:0007bf70+ BLASTER_DSP4xx_BeginPlayback_
0001:0007c010  BLASTER_BeginBufferedPlayback_
0001:0007c09c+ BLASTER_DSP4xx_BeginRecord_
0001:0007c0e4+ BLASTER_DSP2xx_BeginRecord_
0001:0007c168+ BLASTER_DSP1xx_BeginRecord_
0001:0007c1a8  BLASTER_BeginBufferedRecord_
0001:0007c234+ BLASTER_WriteMixer_
0001:0007c250+ BLASTER_ReadMixer_
0001:0007c26c  BLASTER_GetVoiceVolume_
0001:0007c310  BLASTER_SetVoiceVolume_
0001:0007c3bc  BLASTER_GetMidiVolume_
0001:0007c460  BLASTER_SetMidiVolume_
0001:0007c50c  BLASTER_CardHasMixer_
0001:0007c514* BLASTER_SaveVoiceVolume_
0001:0007c588* BLASTER_RestoreVoiceVolume_
0001:0007c5f8  BLASTER_SaveMidiVolume_
0001:0007c66c  BLASTER_RestoreMidiVolume_
0001:0007c6dc  BLASTER_GetEnv_
0001:0007c860  BLASTER_SetCardSettings_
0001:0007c8e0  BLASTER_GetCardSettings_
0001:0007c930  BLASTER_GetCardInfo_
0001:0007c968* BLASTER_SetCallBack_
0001:0007c974+ BLASTER_UnlockMemory_
0001:0007cb2c+ BLASTER_LockMemory_
0001:0007cdd8  BLASTER_SetupWaveBlaster_
0001:0007ce1c  BLASTER_ShutdownWaveBlaster_
0001:0007ce48  BLASTER_Init_
0001:0007d0c8  BLASTER_Shutdown_
0003:00007eb8+ _BLASTER_ErrorCode
Module: audio_wf.lib(D:\PRG\AUDIO\source\pas16.c)
0003:0020a50c+ _PAS_CallBack
0003:0020a514+ _PAS_SoundPlaying
0003:0020a518  _PAS_DMAChannel
0001:0007d220  PAS_ErrorString_
0001:0007d28c+ PAS_CheckForDriver_
0001:0007d310+ PAS_GetStateTable_
0001:0007d364+ PAS_GetFunctionTable_
0001:0007d3b8+ PAS_GetCardSettings_
0001:0007d494+ PAS_EnableInterrupt_
0001:0007d538+ PAS_DisableInterrupt_
0001:0007d60c+ PAS_ServiceInterrupt_
0001:0007d6fc* PAS_Write_
0001:0007d70c+ PAS_Read_
0001:0007d71c+ PAS_SetSampleRateTimer_
0001:0007d7a4+ PAS_SetSampleBufferCount_
0001:0007d830+ PAS_SetPlaybackRate_
0001:0007d898  PAS_GetPlaybackRate_
0001:0007d8a0  PAS_SetMixMode_
0001:0007d8d0  PAS_StopPlayback_
0001:0007d938+ PAS_SetupDMABuffer_
0001:0007d9ac  PAS_GetCurrentPos_
0001:0007da18+ PAS_GetFilterSetting_
0001:0007da60+ PAS_BeginTransfer_
0001:0007db38  PAS_BeginBufferedPlayback_
0001:0007dbb4  PAS_BeginBufferedRecord_
0001:0007dc2c+ PAS_CallMVFunction_
0001:0007dc8c  PAS_SetPCMVolume_
0001:0007dcfc  PAS_GetPCMVolume_
0001:0007dd84  PAS_SetFMVolume_
0001:0007ddf0  PAS_GetFMVolume_
0001:0007de64  PAS_GetCardInfo_
0001:0007debc* PAS_SetCallBack_
0001:0007dec4+ PAS_FindCard_
0001:0007dfa4  PAS_SaveMusicVolume_
0001:0007e09c  PAS_RestoreMusicVolume_
0001:0007e0e0* PAS_SaveState_
0001:0007e134* PAS_RestoreState_
0001:0007e2ec  PAS_Init_
0001:0007e594  PAS_Shutdown_
0001:0007e67c+ PAS_UnlockMemory_
0001:0007e834+ PAS_LockMemory_
0003:00007ef0+ _PAS_ErrorCode
Module: audio_wf.lib(D:\PRG\AUDIO\source\sndscape.c)
0003:0020a570+ _SOUNDSCAPE_CallBack
0003:0020a578+ _SOUNDSCAPE_SoundPlaying
0001:0007ea50+ _SOUNDSCAPE_Interrupts
0001:0007ea90+ _SOUNDSCAPE_SampleSize
0001:0007eaec  SOUNDSCAPE_ErrorString_
0001:0007ee68* SOUNDSCAPE_SetPlaybackRate_
0001:0007eeb4  SOUNDSCAPE_GetPlaybackRate_
0001:0007eebc  SOUNDSCAPE_SetMixMode_
0001:0007eedc  SOUNDSCAPE_StopPlayback_
0001:0007ef84  SOUNDSCAPE_GetCurrentPos_
0001:0007f054  SOUNDSCAPE_BeginBufferedPlayback_
0001:0007f11c  SOUNDSCAPE_GetCardInfo_
0001:0007f138* SOUNDSCAPE_SetCallBack_
0001:0007fc10  SOUNDSCAPE_GetMIDIPort_
0001:0007fc20  SOUNDSCAPE_Init_
0001:0007fd18  SOUNDSCAPE_Shutdown_
0003:00007f10  _SOUNDSCAPE_DMAChannel
0003:00007f14+ _SOUNDSCAPE_ErrorCode
Module: audio_wf.lib(D:\PRG\AUDIO\source\guswave.c)
0003:0020a694  _GUSWAVE_Voices
0003:00007f20  _GUSWAVE_Installed
0001:0007ff8c  GUSWAVE_ErrorString_
0001:000802a0* GUSWAVE_VoicePlaying_
0001:000802b0+ GUSWAVE_VoicesPlaying_
0001:0008030c+ GUSWAVE_Kill_
0001:000803b4  GUSWAVE_KillAllVoices_
0001:0008049c* GUSWAVE_SetPitch_
0001:00080508* GUSWAVE_SetPan3D_
0001:000805bc  GUSWAVE_SetVolume_
0001:00080644  GUSWAVE_GetVolume_
0001:00080740* GUSWAVE_VoiceAvailable_
0001:000807c0+ GUSWAVE_GetNextVOCBlock_
0001:00080a1c+ GUSWAVE_GetNextWAVBlock_
0001:00080a74+ GUSWAVE_GetNextDemandFeedBlock_
0001:00080aec+ GUSWAVE_Play_
0001:00080c50* GUSWAVE_PlayVOC_
0001:00080db0* GUSWAVE_PlayWAV_
0001:00080fc4  GUSWAVE_StartDemandFeedPlayback_
0001:000810a0* GUSWAVE_SetReverseStereo_
0001:000810a8* GUSWAVE_GetReverseStereo_
0001:000811a0* GUSWAVE_SetCallBack_
0001:000811a8  GUSWAVE_Init_
0003:00007f34+ _GUSWAVE_ErrorCode
0003:00007f38+ _GUS_Silence8
0003:00008338+ _GUS_Silence16
Module: audio_wf.lib(D:\PRG\AUDIO\source\sndsrc.c)
0003:0020a77c+ _SS_CallBack
0003:0020a784+ _SS_SoundPlaying
0001:00081254  SS_ErrorString_
0001:00081368  SS_StopPlayback_
0001:000813b4* SS_GetCurrentPos_
0001:000813e0  SS_BeginBufferedPlayback_
0001:00081464* SS_GetPlaybackRate_
0001:0008146c  SS_SetMixMode_
0001:00081470* SS_SetPort_
0001:000814c0* SS_SetCallBack_
0001:000814c8+ SS_TestTimer_
0001:000814d0+ SS_TestSoundSource_
0001:00081560+ SS_DetectSoundSource_
0001:00081634  SS_Init_
0001:00081710  SS_Shutdown_
0001:00081748+ SS_UnlockMemory_
0001:0008184c+ SS_LockMemory_
0003:00008758+ _SS_ErrorCode
Module: audio_wf.lib(D:\PRG\AUDIO\source\multivoc.c)
0003:002137d0  _MV_MixDestination
0003:002137d4  _MV_RightChannelOffset
0003:002137e0  _MV_HarshClipTable
0003:002137e4  _MV_LeftVolume
0003:002137f0+ _MV_MixBuffer
0003:0021383c  _MV_MixPosition
0003:00213840  _MV_RightVolume
0001:000819e2  MV_ErrorString_
0001:00081f28+ MV_ServiceGus_
0001:00081f59+ MV_ServiceRightGus_
0001:000824ee  MV_VoicePlaying_
0001:00082517  MV_KillAllVoices_
0001:0008254f  MV_Kill_
0001:000825c0  MV_VoicesPlaying_
0001:000826d2  MV_VoiceAvailable_
0001:0008274a  MV_SetPitch_
0001:000827b7  MV_SetFrequency_
0001:000829a4+ MV_SetVoiceVolume_
0001:000829e8  MV_SetPan_
0001:00082a27  MV_Pan3D_
0001:00082a92  MV_SetReverb_
0001:00082ad1  MV_SetFastReverb_
0001:00082afb  MV_GetMaxReverbDelay_
0001:00082b04  MV_GetReverbDelay_
0001:00082b1c  MV_SetReverbDelay_
0001:00082b55+ MV_SetMixMode_
0001:00082ceb+ MV_StartPlayback_
0001:00082f63+ MV_StopPlayback_
0001:00082fe8  MV_StartRecording_
0001:000830eb  MV_StopRecord_
0001:00083121  MV_StartDemandFeedPlayback_
0001:00083238  MV_PlayRaw_
0001:00083261  MV_PlayLoopedRaw_
0001:00083367  MV_PlayWAV_
0001:0008338e  MV_PlayWAV3D_
0001:00083437  MV_PlayLoopedWAV_
0001:000836b8  MV_PlayVOC3D_
0001:0008375e  MV_PlayVOC_
0001:00083784  MV_PlayLoopedVOC_
0001:000839d6  MV_SetVolume_
0001:00083aaa  MV_GetVolume_
0001:00083ab0  MV_SetCallBack_
0001:00083ab6  MV_SetReverseStereo_
0001:00083abc  MV_GetReverseStereo_
0001:00083ac2+ MV_TestPlayback_
0001:00083bb8  MV_Init_
0001:00083f45  MV_Shutdown_
0001:00084097+ MV_UnlockMemory_
0001:00084306+ MV_LockMemory_
0003:000087b4  _MV_SampleSize
0003:000087b8  _MV_ErrorCode
0003:000087bc+ _leftpage
0003:000087c0+ _rightpage
Module: audio_wf.lib(D:\PRG\AUDIO\source\user.c)
0001:000845f0  USER_CheckParameter_
0001:00084650  USER_GetText_
Module: audio_wf.lib(D:\PRG\AUDIO\source\ll_man.c)
0001:000846c0  LL_AddNode_
0001:000846e8  LL_RemoveNode_
0001:00084748  LL_UnlockMemory_
0001:0008475c  LL_LockMemory_
Module: H:\WATCOM\lib386\dos\clib3r.lib(fprtf)
0001:000847a0  __fprtf_
Module: H:\WATCOM\lib386\dos\clib3r.lib(vsprintf)
0001:00084870  vsprintf_
Module: H:\WATCOM\lib386\dos\clib3r.lib(dosret)
0001:00084890  _dosret0_
0001:000848a0  _dosretax_
0001:000848b0  __set_errno_dos_
Module: H:\WATCOM\lib386\dos\clib3r.lib(initrtns)
0001:00084940  __InitRtns
0001:00084990  __FiniRtns
Module: H:\WATCOM\lib386\dos\clib3r.lib(allocfp)
0001:000849f0  __allocfp_
0001:00084ab0  __freefp_
0001:00084af0  __purgefp_
Module: H:\WATCOM\lib386\dos\clib3r.lib(ftell)
0001:00084b20  ftell_
Module: H:\WATCOM\lib386\dos\clib3r.lib(_clse)
0001:00084b70  __close_
Module: H:\WATCOM\lib386\dos\clib3r.lib(flush)
0001:00084bc0  __flush_
Module: mact\mact386.lib(joystick.asm)
0003:000087d8  _Joy_x1
0003:000087dc  _Joy_y1
0003:000087e0  _Joy_x2
0003:000087e4  _Joy_y2
0003:000087e8  _Joy_mask
0002:00000000  JoyStick_Vals_
Module: H:\WATCOM\lib386\dos\clib3r.lib(fputs)
0001:00084cd0  fputs_
Module: H:\WATCOM\lib386\dos\clib3r.lib(fputc)
0001:00084d60  fputc_
Module: H:\WATCOM\lib386\dos\clib3r.lib(errno)
0001:00084e30  __get_errno_ptr_
0001:00084e40  __get_doserrno_ptr_
0003:00213860+ _errno
0003:00213864+ __doserrno
Module: H:\WATCOM\lib386\dos\clib3r.lib(strerror)
0001:00084e50  strerror_
0001:00084e70* _strerror_
0003:000087ec+ __sys_nerr
0003:000087f0+ __sys_errlist
Module: H:\WATCOM\lib386\dos\clib3r.lib(accss)
0001:00084f40  access_
Module: H:\WATCOM\lib386\dos\clib3r.lib(getenv)
0001:00084f80  getenv_
Module: H:\WATCOM\lib386\dos\clib3r.lib(chdir)
0001:00084ff0  chdir_
Module: H:\WATCOM\lib386\dos\clib3r.lib(dosdrive)
0001:00085012  _dos_getdrive_
0001:00085026  _dos_setdrive_
Module: audio_wf.lib(D:\PRG\AUDIO\source\awe32.c)
0001:00085060  AWE32_ErrorString_
0001:000850b0  AWE32_NoteOff_
0001:00085108  AWE32_NoteOn_
0001:00085160  AWE32_PolyAftertouch_
0001:00085198  AWE32_ChannelAftertouch_
0001:000851c4  AWE32_ControlChange_
0001:00085258  AWE32_ProgramChange_
0001:00085284  AWE32_PitchBend_
0001:00085698  AWE32_Init_
0001:00085904  AWE32_Shutdown_
0003:000089c0+ _AWE32_ErrorCode
Module: audio_wf.lib(D:\PRG\AUDIO\source\gus.c)
0001:000859eb  GUS_ErrorString_
0001:00085ad3+ D32DosMemAlloc_
0001:00085b3a  GUS_Init_
0001:00085c58  GUS_Shutdown_
0001:00085c97  GUSWAVE_Shutdown_
0003:000089cc  _GUS_AuxError
0003:000089d0  _GUS_ErrorCode
0003:00213a78  _GUS_HoldBuffer
0003:00213a80  _GUS_MemConfig
0003:00213a84+ _GUS_TotalMemory
Module: audio_wf.lib(D:\PRG\AUDIO\source\midi.c)
0003:00213ac8  _MIDI_PatchMap
0001:000867d4  MIDI_RerouteMidiChannel_
0001:000867e8+ MIDI_AllNotesOff_
0001:000868cc  MIDI_SetUserChannelVolume_
0001:00086904  MIDI_ResetUserChannelVolume_
0001:00086960+ MIDI_Reset_
0001:00086a18  MIDI_SetVolume_
0001:00086a98  MIDI_GetVolume_
0001:00086ac4  MIDI_SetContext_
0001:00086ad4  MIDI_GetContext_
0001:00086adc  MIDI_SetLoopFlag_
0001:00086ae4  MIDI_ContinueSong_
0001:00086af8  MIDI_PauseSong_
0001:00086b14  MIDI_SongPlaying_
0001:00086b1c  MIDI_SetMidiFuncs_
0001:00086b24  MIDI_StopSong_
0001:00086ba8  MIDI_PlaySong_
0001:00086e70* MIDI_SetTempo_
0001:00086eb8* MIDI_GetTempo_
0001:000871a0  MIDI_SetSongTick_
0001:00087220  MIDI_SetSongTime_
0001:000872cc  MIDI_SetSongPosition_
0001:00087384  MIDI_GetSongPosition_
0001:000873e8  MIDI_GetSongLength_
0001:00087adc+ MIDI_LoadTimbres_
0001:00087c50+ MIDI_UnlockMemory_
0001:00087e08* MIDI_LockMemory_
0003:00008a80+ _MIDI_Tempo
Module: audio_wf.lib(D:\PRG\AUDIO\source\al_midi.c)
0001:00088010+ AL_SendOutputToPort_
0001:0008804c+ AL_SendOutput_
0001:00088ac4+ AL_FlushCard_
0001:00088be4+ AL_StereoOn_
0001:00088c40+ AL_StereoOff_
0001:00088c8c+ AL_Reset_
0001:00088cfc* AL_ReserveVoice_
0001:00088da4* AL_ReleaseVoice_
0001:00088e18  AL_NoteOff_
0001:00088f5c  AL_NoteOn_
0001:0008903c* AL_AllNotesOff_
0001:0008907c  AL_ControlChange_
0001:00089224  AL_ProgramChange_
0001:00089244  AL_SetPitchBend_
0001:000892c8  AL_DetectFM_
0001:000893ac  AL_Shutdown_
0001:000894e4  AL_SetMaxMidiChannel_
0001:000894ec  AL_Init_
0001:0008970c  AL_RegisterTimbreBank_
Module: audio_wf.lib(D:\PRG\AUDIO\source\mpu401.c)
0001:000897a0+ MPU_SendMidi_
0001:000897d8  MPU_NoteOff_
0001:000897ec  MPU_NoteOn_
0001:00089800  MPU_PolyAftertouch_
0001:00089814  MPU_ControlChange_
0001:0008982c  MPU_ProgramChange_
0001:0008983c  MPU_ChannelAftertouch_
0001:0008984c  MPU_PitchBend_
0001:00089864+ MPU_SendCommand_
0001:00089894  MPU_Reset_
0001:000898d8+ MPU_EnterUART_
0001:0008991c  MPU_Init_
0001:0008995c* MPU_UnlockMemory_
0001:0008998c* MPU_LockMemory_
0003:00009160+ _MPU_BaseAddr
0003:00009164+ _MPU_Delay
Module: audio_wf.lib(D:\PRG\AUDIO\source\gusmidi.c)
0001:000899fd+ GUS_GetPatchMap_
0001:00089c0d+ GUSMIDI_UnloadPatch_
0001:00089cc3+ GUSMIDI_LoadPatch_
0001:00089e47  GUSMIDI_ProgramChange_
0001:00089eb1  GUSMIDI_NoteOn_
0001:00089f3f  GUSMIDI_NoteOff_
0001:00089f70  GUSMIDI_ControlChange_
0001:00089fa4  GUSMIDI_PitchBend_
0001:00089fd8+ GUSMIDI_ReleasePatches_
0001:0008a01d  GUSMIDI_SetVolume_
0001:0008a08e  GUSMIDI_GetVolume_
0001:0008a0ba  GUSMIDI_Init_
0001:0008a1e6  GUSMIDI_Shutdown_
0003:000091c9  _GUSMIDI_Installed
Module: H:\WATCOM\lib386\dos\clib3r.lib(comtflag)
0001:0008a220* __set_commode_
0003:000091d0  __commode
Module: H:\WATCOM\lib386\dos\clib3r.lib(seterrno)
0001:0008a230  __set_errno_
0001:0008a240* __set_EDOM_
0001:0008a250  __set_ERANGE_
0001:0008a260* __set_EINVAL_
0001:0008a270  __set_doserrno_
Module: H:\WATCOM\lib386\dos\clib3r.lib(chktty)
0001:0008a280  __chktty_
Module: H:\WATCOM\lib386\dos\clib3r.lib(int386xa)
0001:0008a2b6  __int386x_
0001:0008a312  _DoINTR_
Module: H:\WATCOM\lib386\dos\clib3r.lib(iomode)
0003:000091d4  ___NFiles
0003:000091d8+ ___init_mode
0001:0008a6a0+ __grow_iomode_
0001:0008a760+ __shrink_iomode_
0001:0008a7a0  __GetIOMode_
0001:0008a810* __IOMode_
0001:0008a820  __SetIOMode_
Module: H:\WATCOM\lib386\dos\clib3r.lib(isatt)
0001:0008a890  isatty_
Module: H:\WATCOM\lib386\dos\clib3r.lib(umaskval)
0003:0000922c  ___umaskval
Module: mact\mact386.lib(P:\LIBMACT\debug.c)
0001:0008a8b0+ DBG_ScreenPrint_
0001:0008a8c0+ DBG_FileStartup_
0001:0008a8f0+ DBG_FilePrint_
0001:0008a914+ DBG_FileShutdown_
0001:0008a934+ DBG_CloseDebugOutput_
0001:0008a958+ DBG_StartDebugOutput_
0001:0008a97c* DBG_SetDebugLevel_
0001:0008a984* DBG_GetDebugLevel_
0001:0008a98c* DBG_EnableDebugLevel_
0001:0008a998* DBG_DisableDebugLevel_
0001:0008a9a4* DBG_DisableAllDebugLevels_
0001:0008a9bc* DBG_SetDebugMode_
0001:0008a9c4* DBG_GetDebugMode_
0001:0008a9cc* DBG_SetDebugOutputMode_
0001:0008aa18* DBG_GetDebugOutputMode_
0001:0008aa20* DBG_DebugString_
0001:0008ab10  DBG_DbgString_
0001:0008ac00* DBG_Shutdown_
0001:0008ac3c* DBG_Startup_
0001:0008ac98* DBG_RegisterOutputFunction_
Module: H:\WATCOM\lib386\dos\clib3r.lib(vprintf)
0001:0008acc0  vprintf_
Module: H:\WATCOM\lib386\dos\clib3r.lib(nmsize)
0001:0008ace0  _msize_
0001:0008acf0  _nmsize_
Module: H:\WATCOM\lib386\dos\clib3r.lib(nrealloc)
0001:0008ad00  realloc_
0001:0008ad10+ _nrealloc_
Module: H:\WATCOM\lib386\dos\clib3r.lib(qwrit)
0001:0008adb0  __qwrite_
Module: H:\WATCOM\lib386\dos\clib3r.lib(ioalloc)
0001:0008ae30  __ioalloc_
Module: H:\WATCOM\lib386\dos\clib3r.lib(tell)
0001:0008aed0  tell_
Module: H:\WATCOM\lib386\dos\clib3r.lib(cmain386)
0001:0008aef0  __CMain
Module: H:\WATCOM\lib386\dos\clib3r.lib(dosseg)
0000:00001234  __DOSseg__
Module: H:\WATCOM\lib386\dos\clib3r.lib(crwdata)
0003:00009303  __osmajor
0003:00009304  __osminor
0003:000092d8  __psp
0003:000092fa  __Extender
0003:000092fb  __ExtenderSubtype
0003:000092fc  __X32VM
0003:000092dc* __x386_stacklow
0003:000092d0  __LpCmdLine
0003:000092d4  __LpPgmName
0003:000092c8  __dynend
0003:000092cc  __curbrk
0003:000092dc  __STACKLOW
0003:000092e0  __STACKTOP
0003:000092e4  __ASTACKSIZ
0003:000092e8  __ASTACKPTR
0003:000092ec  __cbyte
0003:000092f0* __cbyte2
0003:000092f4  __child
0003:000092fd  __Envptr
0003:00009301  __Envseg
0003:000092f8  __no87
0003:00009305  __FPE_handler
0003:00009305  ___FPE_handler
Module: H:\WATCOM\lib386\dos\clib3r.lib(initargv)
0001:0008af30  __Init_Argv_
0001:0008b170  __Fini_Argv_
Module: H:\WATCOM\lib386\dos\clib3r.lib(doserror)
0001:0008b186  __doserror_
Module: H:\WATCOM\lib386\dos\clib3r.lib(nmemneed)
0001:0008b1a0  __nmemneed_
Module: H:\WATCOM\lib386\dos\clib3r.lib(mem)
0001:0008b1b0  __MemAllocator
0001:0008b270  __MemFree
Module: H:\WATCOM\lib386\dos\clib3r.lib(grownear)
0001:0008b440+ __FreeDPMIBlocks_
0001:0008b4b0  __ReAllocDPMIBlock_
0001:0008b640+ __LastFree_
0001:0008b840  __ExpandDGROUP_
Module: H:\WATCOM\lib386\dos\clib3r.lib(heapmod)
0003:00218080  ___nheap_clean
0003:00218081  ___fheap_clean
Module: H:\WATCOM\lib386\dos\clib3r.lib(xmsg)
0001:0008ba10+ __exit_with_msg_
0001:0008ba20  __fatal_runtime_error_
Module: H:\WATCOM\lib386\dos\clib3r.lib(__stos)
0001:0008ba40  __STOSB
0001:0008ba77  __STOSD
Module: H:\WATCOM\lib386\dos\clib3r.lib(gtctm)
0001:0008baf0  __getctime_
Module: H:\WATCOM\lib386\dos\clib3r.lib(mktime)
0001:0008bbd0  mktime_
Module: H:\WATCOM\lib386\dos\clib3r.lib(initfile)
0001:0008bd60  __InitFiles_
Module: H:\WATCOM\lib386\dos\clib3r.lib(ioexit)
0001:0008be00  __full_io_exit_
0001:0008be10* fcloseall_
Module: H:\WATCOM\lib386\dos\clib3r.lib(flushall)
0001:0008be80  flushall_
0001:0008be90  __flushall_
Module: mact\mact386.lib(P:\LIBMACT\tokenlib.c)
0001:0008bed0* TOKEN_GetLineNumber_
0001:0008befc  TOKEN_Reset_
0001:0008bf54* SkipToEOL_
0001:0008bf74+ TOKEN_CheckOverflow_
0001:0008bfb4+ TOKEN_SkipWhiteSpace_
0001:0008c03c+ TOKEN_SkipNonToken_
0001:0008c0b0+ TOKEN_TokenAvailable_
0001:0008c184  TOKEN_CommentAvailable_
0001:0008c1f0* TOKEN_UnGet_
0001:0008c220+ TOKEN_Get_
0001:0008c2d8+ TOKEN_GetLine_
0001:0008c3a0  TOKEN_GetRaw_
0001:0008c450* TOKEN_GetSpecific_
0001:0008c4a4* TOKEN_GetInteger_
0001:0008c4dc* TOKEN_GetDouble_
0001:0008c514* TOKEN_LinesInFile_
0001:0008c5ac+ TOKEN_New_
0001:0008c614  TOKEN_Free_
0001:0008c654  TOKEN_Parse_
0001:0008c6e4* TOKEN_Load_
0003:002180e0  _token
Module: H:\WATCOM\lib386\dos\clib3r.lib(sscanf)
0001:0008c750+ vsscanf_
0001:0008c780  sscanf_
Module: H:\WATCOM\lib386\dos\clib3r.lib(fltused)
0003:00009310  _fltused_
Module: H:\WATCOM\lib386\dos\emu387.lib(386)
0001:0008c7b0  __init_387_emulator
0001:0008c7b5* __fini_387_emulator
Module: H:\WATCOM\lib386\dos\clib3r.lib(01h)
0003:00009314  __8087
0003:00009315  __real87
Module: H:\WATCOM\lib386\dos\clib3r.lib(qread)
0001:0008c7c0  __qread_
Module: H:\WATCOM\lib386\dos\clib3r.lib(fgetc)
0001:0008c7f0  fgetc_
0001:0008c8a0+ __filbuf_
0001:0008c8d0  __fill_buffer_
Module: H:\WATCOM\lib386\dos\clib3r.lib(bits)
0001:0008c9b0  __setbits_
0003:000068cc  __Bits
Module: audio_wf.lib(D:\PRG\AUDIO\source\dma.c)
0001:0008cb00  DMA_ErrorString_
0001:0008cb48  DMA_VerifyChannel_
0001:0008cb90  DMA_SetupTransfer_
0001:0008cc98  DMA_EndTransfer_
0001:0008cccc  DMA_GetCurrentPos_
0001:0008cd28* DMA_GetTransferCount_
0003:00009318+ _DMA_ErrorCode
Module: audio_wf.lib(D:\PRG\AUDIO\source\irq.c)
0001:0008cde8* rmcallback_
0001:0008ce78  IRQ_SetVector_
0001:0008d090  IRQ_RestoreVector_
Module: H:\WATCOM\lib386\dos\clib3r.lib(rewind)
0001:0008d160  rewind_
Module: H:\WATCOM\lib386\dos\clib3r.lib(fgets)
0001:0008d180  fgets_
Module: H:\WATCOM\lib386\dos\clib3r.lib(strstr)
0001:0008d200  strstr_
Module: H:\WATCOM\lib386\dos\clib3r.lib(strtol)
0001:0008d490* strtoul_
0001:0008d4a0  strtol_
Module: audio_wf.lib(D:\PRG\AUDIO\source\debugio.c)
0001:0008d510* DB_SetXY_
0001:0008d524+ DB_PutChar_
0001:0008d5fc+ DB_PrintString_
0001:0008d680  DB_PrintNum_
0001:0008d6cc* DB_PrintUnsigned_
0001:0008d700  DB_printf_
Module: audio_wf.lib(C:\PRG\NEWGF1\GF1NEW\digital.c)
0003:002181a0+ _dig_voice_status
0001:0008d810  dig_init_
0001:0008d94c+ dig_change_voice_
0001:0008daa0+ gf1_restart_digital_
0001:0008dd8c  gf1_dig_set_vol_
0001:0008ddec  gf1_dig_set_pan_
0001:0008df0c  gf1_dig_set_freq_
0001:0008df50  gf1_stop_digital_
0001:0008e210+ gf1_start_digital_
0001:0008e31c* gf1_dig_set_dma_rate_
0001:0008e32c+ dig_dma_next_buffer_
0001:0008e954+ gf1_play_next_buffer_
0001:0008e9c4  gf1_play_digital_
Module: audio_wf.lib(D:\PRG\AUDIO\source\pitch.c)
0001:0008eba0  PITCH_GetScale_
0001:0008ec50  PITCH_UnlockMemory_
0001:0008ec74  PITCH_LockMemory_
Module: audio_wf.lib(C:\PRG\NEWGF1\GF1NEW\gf1mem.c)
0001:0008ecc0+ gf1_write_block_
0001:0008ecf8  gf1_read_block_
0001:0008ed2c  gf1_mem_init_
0001:0008ede0  gf1_malloc_
0001:0008ef18  gf1_free_
0001:0008effc  gf1_mem_avail_
0001:0008f070* gf1_mem_largest_avail_
Module: audio_wf.lib(.\source\mvreverb.ASM)
0001:0008f12b  MV_8BitReverb_
0001:0008f143  MV_16BitReverbFast_
0001:0008f164  MV_8BitReverbFast_
0001:0008f0f8  MV_16BitReverb_
Module: audio_wf.lib(.\source\mv_mix.ASM)
0001:0008f432  MV_Mix16BitStereo_
0001:0008f270  MV_Mix8BitStereo_
0001:0008f33d  MV_Mix16BitMono_
0001:0008f190  MV_Mix8BitMono_
Module: audio_wf.lib(.\source\mv_mix16.ASM)
0001:0008f518  MV_Mix8BitMono16_
0001:0008f6eb  MV_Mix16BitMono16_
0001:0008f613  MV_Mix8BitStereo16_
0001:0008f7af  MV_Mix16BitStereo16_
Module: H:\WATCOM\lib386\dos\clib3r.lib(prtf)
0001:0008f8f0  __prtf_
Module: H:\WATCOM\lib386\dos\clib3r.lib(sgdef086)
0003:0001107c  __Start_XI
0003:000110c4  __End_XI
0003:000110c4  __Start_YI
0003:000110ee  __End_YI
Module: H:\WATCOM\lib386\dos\clib3r.lib(fsync)
0001:00090770  fsync_
Module: H:\WATCOM\lib386\dos\clib3r.lib(environ)
0003:00219d60  ___env_mask
0003:00219d64  _environ
0003:00219d68* __wenviron
Module: H:\WATCOM\lib386\dos\clib3r.lib(mbsnicmp)
0001:00090780  _mbsnicmp_
Module: audio_wf.lib(midieng.c)
0001:00090804  ___midieng_code
0001:0009080c  AWE32INITMIDI
0001:00091ffc  AWE32PROGRAMCHANGE
0001:000908b4  AWE32REGW
0001:0009091c  AWE32REGRW
0001:00090984  AWE32REGDW
0001:000909fc  AWE32REGRDW
0001:00090a70  ___awe32AllocGChannel
0001:000916e4  AWE32NOTEOFF
0001:00091804  AWE32NOTEON
0001:00091cdc  AWE32CONTROLLER
0001:000921b4  AWE32POLYKEYPRESSURE
0001:000921bc  AWE32CHANNELPRESSURE
0001:00092204  AWE32PITCHBEND
0001:000923f0* AWE32SYSEX
0001:00092470  ___midieng_ecode
Module: audio_wf.lib(embed.c)
0003:00009e30  ___embed_data
0003:00009e34  _awe32SPad1Obj
0003:0000a03c  _awe32SPad2Obj
0003:0000a1a8  _awe32SPad3Obj
0003:0000a71c  _awe32SPad4Obj
0003:0000a884  _awe32SPad5Obj
0003:0000ae50  _awe32SPad6Obj
0003:0000d8d0  _awe32SPad7Obj
0003:0000e250  ___embed_edata
Module: audio_wf.lib(sbkload.c)
0001:00092478* ___sbkload_code
0001:00092480  AWE32TOTALPATCHRAM
0001:00092494  AWE32DEFINEBANKSIZES
0001:00092554* AWE32RELEASEBANK
0001:000925ec* AWE32RELEASEALLBANKS
0001:00092ad0* AWE32SETPRESETS
0001:00093114* AWE32STREAMSAMPLE
0001:0009317c* AWE32SFONTLOADREQUEST
0001:000932f4* AWE32WPLOADREQUEST
0001:000933a0* AWE32WPLOADWAVE
0001:00093414* AWE32WPSTREAMWAVE
0001:000934bc* AWE32WPBUILDSFONT
0001:00093644* __AWE32NOTEOFF
0001:000936dc* __AWE32ISPLAYING
0001:00093784* ___sbkload_ecode
Module: audio_wf.lib(midivar.c)
0003:0000e45c  ___midivar_data
0003:0000e460  _awe32NumG
0003:0000e462  _awe32BaseAddx
0003:0000e464  _awe32DramSize
0003:0000e468  _awe32Scratch
0003:0000e728  _awe32SFont
0003:0000e918  _awe32GChannel
0003:0000eb98  _awe32MIDIChannel
0003:0000ed98  _awe32SoundPad
0003:0000edb4  ___midivar_edata
Module: audio_wf.lib(hardware.c)
0001:0009378c* ___hardware_code
0001:00093794  AWE32DETECT
0001:00094034  AWE32INITHARDWARE
0001:0009417c  AWE32TERMINATE
0001:000941e8* ___hardware_ecode
Module: audio_wf.lib(nrpn.c)
0001:000941f0  ___nrpn_code
0001:000941f8  AWE32INITNRPN
0001:00094ce0  ___nrpn_ecode
Module: audio_wf.lib(nrpnvar.c)
0003:0000f204  ___nrpnvar_data
0003:0000f208  _awe32NRPNChannel
0003:0000f808  ___nrpnvar_edata
Module: audio_wf.lib(C:\PRG\NEWGF1\GF1NEW\gf1error.c)
0001:00094d3c  gf1_error_str_
Module: audio_wf.lib(C:\PRG\NEWGF1\GF1NEW\gf1utils.c)
0001:00094e10  GetUltraCfg_
Module: audio_wf.lib(C:\PRG\NEWGF1\GF1NEW\gf1init.c)
0001:00095040+ gf1_initialize_
0001:000950ec+ gf1_ramp_down_
0001:00095298  gf1_load_os_
0001:00095384  gf1_unload_os_
0001:0009557c+ reset_ultra_
0003:00219d80* _old_gf1_service
0003:00219d86* _old_midi_service
Module: audio_wf.lib(D:\PRG\AUDIO\source\gmtimbre.c)
0003:0000f824  _ADLIB_TimbreBank
Module: H:\WATCOM\lib386\dos\clib3r.lib(strcat)
0001:000958b0  strcat_
Module: audio_wf.lib(C:\PRG\NEWGF1\GF1NEW\gf1patch.c)
0001:000958f0  gf1_get_patch_info_
0001:000959d8  gf1_load_patch_
0001:00095e6c  gf1_unload_patch_
0001:00095ef8* gf1_detune_patch_
Module: audio_wf.lib(C:\PRG\NEWGF1\GF1NEW\gf1note.c)
0001:00095f10  gf1_note_init_
0001:000963f8  gf1_midi_change_volume_
0001:00096480  gf1_channel_pitch_bend_
0001:0009655c  gf1_midi_synth_volume_
0001:00096608  gf1_midi_set_vibrato_
0001:00096b78+ gf1_calc_fc_
0001:00096c30+ gf1_midi_stop_voice_
0001:00096d74+ gf1_midi_status_voice_
0001:00096e14* gf1_midi_status_note_
0001:00096e64+ gf1_midi_wait_voice_
0001:00096f60+ gf1_midi_stop_note_
0001:00096fd4  gf1_midi_note_on_
0001:0009765c  gf1_midi_note_off_
0001:00097b60  gf1_midi_channel_sustain_
0001:0009807c  gf1_midi_silence_patch_notes_
0001:0009818c  gf1_midi_patch_removed_
0001:000981b8  gf1_midi_change_program_
0001:000981d4  gf1_midi_set_balance_
0001:00098280* gf1_midi_all_sounds_off_
0001:000982f8  gf1_midi_all_notes_off_
0003:00010524  _gf1_log_table
0003:00010554+ _gf1_linear_volumes
0003:00219d90+ _voice_status
0003:0021a1b0+ _other_voices
0003:0021a2b0+ _note_status
0003:0021a330+ _channel_status
0003:0021a570+ _gf1_m_volume
0003:0021a574+ _vibrato_voice_count
Module: audio_wf.lib(C:\PRG\NEWGF1\GF1NEW\gf1midi.c)
0001:00098350  gf1_midi_pitch_bend_
0001:00098438  gf1_midi_parameter_
0003:00010558+ _pbs_msb
0003:00010598+ _pbs_lsb
0003:000105d8+ _rpn_msb
0003:00010618+ _rpn_lsb
0003:00010658+ _channel_volume
0003:00010698+ _channel_expression
0003:000106d8* _channel_pan
Module: H:\WATCOM\lib386\dos\clib3r.lib(nexpand)
0001:000986c0* _expand_
0001:000986d0+ __HeapManager_expand_
0001:000988b0  _nexpand_
Module: H:\WATCOM\lib386\dos\clib3r.lib(cinit)
0001:00098930  __CommonInit_
Module: H:\WATCOM\lib386\dos\clib3r.lib(___argc)
0003:0021a580  ____Argc
0003:0021a584  ____Argv
Module: H:\WATCOM\lib386\dos\clib3r.lib(histsplt)
0003:0021a588  ___historical_splitparms
Module: H:\WATCOM\lib386\dos\clib3r.lib(heapen)
0001:000989a0* _heapenable_
0003:00010718  ___heap_enabled
Module: H:\WATCOM\lib386\dos\clib3r.lib(minreal)
0003:0021a590  ___minreal
Module: H:\WATCOM\lib386\dos\clib3r.lib(sbrk386)
0001:000989b0* sbrk_
0001:00098a90  __brk_
Module: H:\WATCOM\lib386\dos\clib3r.lib(amblksiz)
0003:0001071c  __amblksiz
Module: H:\WATCOM\lib386\dos\clib3r.lib(enterdb)
0001:00098bb0  __EnterWVIDEO_
0003:00010720+ ___WD_Present
Module: H:\WATCOM\lib386\dos\clib3r.lib(timeutil)
0001:00098be0  __leapyear_
0001:00098d70  __isindst_
0003:000068d4  ___diyr
0003:000068ee  ___dilyr
Module: H:\WATCOM\lib386\dos\clib3r.lib(gmtime)
0001:00099110  __brktime_
0001:00099230+ _gmtime_
0001:00099250* gmtime_
Module: H:\WATCOM\lib386\dos\clib3r.lib(tzset)
0003:00010724  ___start_dst
0003:00010748  ___end_dst
0003:00010870* _tzname
0003:00010878  _timezone
0003:0001087c  _daylight
0003:00010880  ___dst_adjust
0001:00099260* __DontCacheOSTZ_
0001:00099280* __CacheOSTZ_
0001:000992d0  tzset_
0001:00099540+ __parse_tz_
Module: H:\WATCOM\lib386\dos\clib3r.lib(atoi)
0001:00099660  atoi_
Module: H:\WATCOM\lib386\math387r.lib(strtod)
0001:000996a9+ __Strtold_
0001:00099878  strtod_
Module: H:\WATCOM\lib386\dos\clib3r.lib(scnf)
0001:00099990  __scnf_
Module: H:\WATCOM\lib386\dos\clib3r.lib(setefg)
0001:0009a930  __setEFGfmt_
Module: H:\WATCOM\lib386\math387r.lib(dosinite)
0001:0009a94c  __sys_init_387_emulator
0001:0009aad1  __sys_fini_387_emulator
Module: H:\WATCOM\lib386\dos\clib3r.lib(chk8087)
0001:0009abd0+ __init_8087_
0001:0009ac10* _fpreset_
0001:0009ac20  __chk8087_
Module: H:\WATCOM\lib386\dos\clib3r.lib(gtche)
0001:0009ac70  getche_
Module: audio_wf.lib(wdigital.asm)
0003:000108d4  _dig_init_data
Module: audio_wf.lib(C:\PRG\NEWGF1\GF1NEW\globals.c)
0003:000108d8  _gf1_pstatus
0003:000108dc  _gf1_mix_control
0003:000108de  _gf1_status_register
0003:000108e0  _gf1_timer_control
0003:000108e2  _gf1_timer_data
0003:000108e4  _gf1_irqdma_control
0003:000108e6  _gf1_reg_control
0003:000108e8  _gf1_midi_control
0003:000108ea  _gf1_midi_data
0003:000108ec  _gf1_page_register
0003:000108ee  _gf1_register_select
0003:000108f0  _gf1_data_low
0003:000108f2  _gf1_data_high
0003:000108f4  _gf1_dram_io
0003:000108f6  _gf1_dma_latch
0003:0021a5d0  _gf1_voices
0003:0021a5d2  _gf1_flags
0003:0021a5d4  _gf1_semaphore
0003:0021a5d6  _gf1_status
0003:0021a5d8  _mixer_mask
0003:0021a5d9  _gf1_channel_out
0003:0021a5da  _gf1_channel_in
0003:0021a5db  _midi_irq
0003:0021a5dc  _gf1_irq
Module: audio_wf.lib(C:\PRG\NEWGF1\GF1NEW\gf1isr.c)
0003:00010904  _visr
0001:0009ac90  gf1_isr_init_
0001:0009ad3c  gf1_add_dma_handler_
0001:0009ad74  gf1_add_voice_handler_
0001:0009adac  gf1_add_volume_handler_
0001:0009ade4  gf1_add_timer_handler_
0001:0009ae28  gf1_add_midi_recv_handler_
0001:0009ae48* gf1_add_midi_xmit_handler_
0001:0009ae68  gf1_add_visr_
0001:0009ae88  process_midi_interrupt_
0001:0009af40  process_interrupt_
0003:0021a5e0  _gf1_adlib_control
Module: audio_wf.lib(C:\PRG\NEWGF1\GF1NEW\gf1addr.c)
0001:0009b1e0  convert_to_16bit_
0001:0009b1fc* make_physical_address_
0001:0009b258  gf1_set_addr_regs_
Module: H:\WATCOM\lib386\dos\clib3r.lib(outp)
0001:0009b2f0  outp_
Module: audio_wf.lib(gf1init2.asm)
0001:0009b301  gf1_delay_
0001:0009b315  gf1_init_ports_
Module: audio_wf.lib(gf1sem.asm)
0001:0009b360  gf1_init_semaphores_
0001:0009b373  gf1_enter1_
0001:0009b39a  gf1_leave_
0001:0009b37b* gf1_enter_
0003:00010934* _num_sems
Module: H:\WATCOM\lib386\dos\clib3r.lib(inpw)
0001:0009b3d0  inpw_
Module: H:\WATCOM\lib386\dos\clib3r.lib(inp)
0001:0009b3e0  inp_
Module: audio_wf.lib(C:\PRG\NEWGF1\GF1NEW\divisor.c)
0003:0001094c  _gf1_freq_divisor
Module: H:\WATCOM\lib386\dos\clib3r.lib(outpw)
0001:0009b3f0  outpw_
Module: audio_wf.lib(C:\PRG\NEWGF1\GF1NEW\gf1dma.c)
0001:0009b44c  gf1_dma_init_
0001:0009b55c  gf1_dram_xfer_
0001:0009b798  gf1_wait_dma_
0001:0009b81c  gf1_dma_ready_
0001:0009b834  gf1_stop_dma_
0003:0021a5f0+ _dma_parms
Module: audio_wf.lib(C:\PRG\NEWGF1\GF1NEW\gf1voice.c)
0001:0009b8d0  gf1_voice_init_
0001:0009b91c  gf1_allocate_voice_
0001:0009ba74  gf1_free_voice_
0001:0009baac  gf1_adjust_priority_
Module: audio_wf.lib(C:\PRG\NEWGF1\GF1NEW\gf1dram.c)
0001:0009bae0  gf1_peek_
0001:0009bb5c  gf1_poke_
0001:0009bbdc  gf1_poke_block_
0001:0009bcc8  gf1_good_dram_
Module: audio_wf.lib(gf1wmem.asm)
0003:0001097c  _gf1_mem_init_data
Module: H:\WATCOM\lib386\dos\clib3r.lib(wctomb)
0001:0009be80  wctomb_
Module: H:\WATCOM\lib386\dos\clib3r.lib(itoa)
0001:0009beb0+ utoa_
0001:0009bf00  itoa_
Module: H:\WATCOM\lib386\dos\clib3r.lib(noefgfmt)
0003:00010980  ___EFG_printf
0003:00010984  ___EFG_scanf
Module: H:\WATCOM\lib386\dos\clib3r.lib(lltoa)
0001:0009bf50  __clib_ulltoa_
0001:0009bfc0* __clib_lltoa_
Module: H:\WATCOM\lib386\dos\clib3r.lib(mbisdbcs)
0003:0021a7a0  ___IsDBCS
Module: H:\WATCOM\lib386\dos\clib3r.lib(mbislead)
0001:0009bff0* _ismbblead_
0003:0021a7b0  ___MBCSIsTable
Module: H:\WATCOM\lib386\dos\clib3r.lib(dosfile)
0001:0009c008  _dos_close_
0001:0009c017  _dos_commit_
0001:0009c027  _dos_open_
Module: H:\WATCOM\lib386\dos\clib3r.lib(setenvp)
0001:0009c050  __setenvp_
0001:0009c170  __freeenvp_
Module: H:\WATCOM\lib386\dos\clib3r.lib(mbterm)
0001:0009c1d0  _mbterm_
Module: H:\WATCOM\lib386\dos\clib3r.lib(mbcicmp)
0001:0009c210  _mbcicmp_
Module: H:\WATCOM\lib386\dos\clib3r.lib(mbsinc)
0001:0009c270  _mbsinc_
Module: audio_wf.lib(C:\PRG\NEWGF1\GF1NEW\os\dos32\watcom\os.c)
0001:0009c2a0  os_init_channel_
0001:0009c32c  os_pgm_dma_
0001:0009c450  os_stop_dma_
0001:0009c478* os_dma_count_
0001:0009c4e0  os_file_read_
0001:0009c510  os_file_close_
0001:0009c52c  os_file_seek_
0001:0009c548  os_file_open_
0001:0009c574+ os_setvect_
0001:0009c580+ os_getvect_
0001:0009c58c  os_set_irq_
0001:0009c624  os_unset_irq_
0001:0009c6a8  os_eoi_
0003:000109a2+ _os_irq_table
Module: audio_wf.lib(C:\PRG\NEWGF1\GF1NEW\gf1wisr.c)
0001:0009c6e0  gf1_irq_service_
0001:0009c75c  midi_irq_service_
Module: audio_wf.lib(C:\PRG\NEWGF1\GF1NEW\gf1detct.c)
0001:0009c7e0  gf1_detect_card_
Module: audio_wf.lib(gf1ainit.asm)
0003:00011112* Gf1InitEnd
0003:000110ee* Gf1InitStart
0001:0009c840  gf1_asm_init_
Module: audio_wf.lib(C:\PRG\NEWGF1\GF1NEW\gf1wave.c)
0001:0009c8b0  gf1_update_waveform_
Module: audio_wf.lib(gf1wnote.asm)
0003:00010a28  _gf1_note_init_data
Module: audio_wf.lib(C:\PRG\NEWGF1\GF1NEW\voltab.c)
0003:00010a2c  _vol_table
Module: audio_wf.lib(C:\PRG\NEWGF1\GF1NEW\timer.c)
0001:0009ca00  gf1_timer_init_
0001:0009ca24  gf1_enable_timer2_
0001:0009cae8* gf1_enable_timer1_
0001:0009cbac* gf1_disable_timer1_
0001:0009cc18  gf1_disable_timer2_
Module: audio_wf.lib(C:\PRG\NEWGF1\GF1NEW\gf1scale.c)
0003:00010aac  _gf1_scale_table
Module: H:\WATCOM\lib386\dos\clib3r.lib(sigsy)
0001:0009cdd0  __DPMI_hosted_
0001:0009ce70  __restore_int23_
0001:0009cf70  __restore_int_ctrl_break_
0001:0009d0b0  __grab_int23_
0001:0009d210  __grab_int_ctrl_break_
Module: H:\WATCOM\lib386\dos\clib3r.lib(bufld386)
0001:0009d3a8  __ZBuf2LD
Module: H:\WATCOM\lib386\math387r.lib(ldcvt)
0001:0009d533  _LDScale10x_
0001:0009d58f  __LDcvt_
Module: H:\WATCOM\lib386\dos\clib3r.lib(hugeval)
0003:00006960  __HugeValue
Module: H:\WATCOM\lib386\dos\clib3r.lib(mbtowc)
0001:0009dff0  mbtowc_
Module: H:\WATCOM\lib386\dos\clib3r.lib(fdfs386)
0001:0009e0ac  __FDFS
Module: H:\WATCOM\lib386\dos\clib3r.lib(i8m)
0001:0009e0f8* __I8M
0001:0009e0f8  __U8M
Module: H:\WATCOM\lib386\math387r.lib(efgfmt)
0001:0009e2af  _EFG_Format_
Module: H:\WATCOM\lib386\math387r.lib(cnvs2d)
0001:0009e4a5  __cnvs2d_
Module: H:\WATCOM\lib386\dos\emu387.lib(emu387)
0001:0009e834* stkop1
0001:0009e874  __int7_pl3
0001:0009e898* __int7_X32VM
0001:0009e8e4  __int7
Module: H:\WATCOM\lib386\dos\clib3r.lib(hook387)
0001:000a1950  __hook387
0001:000a1a00  __unhook387
Module: H:\WATCOM\lib386\dos\clib3r.lib(8087cw)
0003:00010df8  __8087cw
Module: H:\WATCOM\lib386\dos\clib3r.lib(save8087)
0003:00010dfc  ___Save8087
0003:00010e00  ___Rest8087
Module: H:\WATCOM\lib386\dos\clib3r.lib(init8087)
0001:000a1a52  __init_80x87
Module: audio_wf.lib(gf1wdma.asm)
0003:00010e04  _gf1_dma_init_data
Module: audio_wf.lib(gf1wvoic.asm)
0003:00010e06  _gf1_voice_init_data
Module: H:\WATCOM\lib386\dos\clib3r.lib(mbinit)
0001:000a1a80  __mbinit_
0001:000a1bf0+ dos_get_dbcs_lead_table_
0001:000a1d00+ dos_get_code_page_
0003:00010e08  ___MBCodePage
Module: H:\WATCOM\lib386\dos\clib3r.lib(clearenv)
0001:000a1ef0  clearenv_
Module: H:\WATCOM\lib386\dos\clib3r.lib(mbccpy)
0001:000a1f90  _mbccpy_
Module: H:\WATCOM\lib386\dos\clib3r.lib(mbclen)
0001:000a1fd0  _mbclen_
Module: H:\WATCOM\lib386\dos\clib3r.lib(mbsupr)
0001:000a2000  _mbsupr_
Module: H:\WATCOM\lib386\dos\clib3r.lib(mbccmp)
0001:000a2050  _mbccmp_
Module: H:\WATCOM\lib386\dos\clib3r.lib(dosio)
0001:000a20aa  _dos_read_
0001:000a20d4* _dos_write_
Module: audio_wf.lib(wtimer.asm)
0003:00010e0c  _gf1_timer_init_data
Module: H:\WATCOM\lib386\dos\clib3r.lib(signl)
0001:000a20e0+ __sigabort_
0001:000a20f0  __sigfpe_handler_
0001:000a2130* signal_
0001:000a2250  raise_
Module: H:\WATCOM\lib386\dos\clib3r.lib(nonibm)
0001:000a2330+ __is_nonIBM_
0003:00010e44  ___NonIBM
Module: H:\WATCOM\lib386\math387r.lib(ldclass)
0001:000a238b  __LDClass_
Module: H:\WATCOM\lib386\dos\clib3r.lib(intr)
0001:000a23e0  intr_
Module: H:\WATCOM\lib386\dos\clib3r.lib(inirmsel)
0003:0021ad90  __ExtenderRealModeSelector
Module: H:\WATCOM\lib386\dos\clib3r.lib(intd386)
0001:000a2520  intdos_
Module: H:\WATCOM\lib386\dos\clib3r.lib(mbsnextc)
0001:000a2570  _mbsnextc_
Module: H:\WATCOM\lib386\dos\clib3r.lib(mbcupper)
0001:000a25b0  _mbctoupper_
Module: H:\WATCOM\lib386\dos\clib3r.lib(mbconv)
0001:000a2620  _mbvtop_
Module: H:\WATCOM\lib386\dos\clib3r.lib(abort)
0001:000a2640* abort_
0001:000a2650  __terminate_
0003:00010e48  ___abort
Module: H:\WATCOM\lib386\dos\clib3r.lib(cntrl87)
0001:000a2670  _control87_
Module: H:\WATCOM\lib386\math387r.lib(grabfpe)
0001:000a26ca  __grab_fpe_
Module: H:\WATCOM\lib386\dos\clib3r.lib(mbdtoupp)
0001:000a26d0  _mbdtoupper_
Module: H:\WATCOM\lib386\dos\clib3r.lib(grabfp87)
0001:000a26f0  __GrabFP87_
Module: H:\WATCOM\lib386\dos\clib3r.lib(ismbdlow)
0001:000a2770  _ismbdlower_
Module: H:\WATCOM\lib386\dos\clib3r.lib(fpe387)
0003:00010e4c  ___PMSeg
0003:00010e4e  ___PMAddr
0003:00010e52  ___RMAddr
0001:000a27ae  __Init_FPE_handler_
0001:000a280b  __Fini_FPE_handler_
Module: H:\WATCOM\lib386\dos\clib3r.lib(fpeinth)
0001:000a2868  __Enable_FPE_
0001:000a287d  __FPEHandler_
0001:000a287d  ___FPEHandlerStart_
0001:000a288a  __FPE2Handler_
0001:000a298d  ___FPEHandlerEnd_
Module: H:\WATCOM\lib386\dos\clib3r.lib(mbislegl)
0001:000a2ad0  _ismbclegal_
Module: H:\WATCOM\lib386\dos\clib3r.lib(fpephar)
0001:000a2b10  __Phar_hook_init_
0001:000a2bd3  __Phar_hook_fini_
Module: H:\WATCOM\lib386\dos\clib3r.lib(fpedos4g)
0001:000a2c00  __DOS4G_hook_init_
0001:000a2c2d  __DOS4G_hook_fini_
Module: H:\WATCOM\lib386\dos\clib3r.lib(fpeergo)
0001:000a2c46  __Ergo_hook_init_
0001:000a2c84  __Ergo_hook_fini_
Module: H:\WATCOM\lib386\dos\clib3r.lib(fpeintel)
0001:000a2c9e  __Intel_hook_init_
0001:000a2cf6  __Intel_hook_fini_
Module: H:\WATCOM\lib386\dos\clib3r.lib(mbistrai)
0001:000a2d00  _ismbbtrail_
Module: H:\WATCOM\lib386\dos\clib3r.lib(fpeint)
0003:00011074  ___FPE_int
0003:00011075  ___IRQ_num
0003:00011076  ___IRQ_int
0003:00011077  ___MST_pic
0003:00011078+ ___SLV_pic
Module: H:\WATCOM\lib386\dos\clib3r.lib(isktable)
0003:00006968  __IsKTable


                        +----------------------+
                        |   Imported Symbols   |
                        +----------------------+

Symbol                              Module
======                              ======



                        +--------------------+
                        |   Libraries Used   |
                        +--------------------+

audio_wf.lib
mact\mact386.lib
H:\WATCOM\lib386\dos\clib3r.lib
H:\WATCOM\lib386\math387r.lib
H:\WATCOM\lib386\dos\emu387.lib


                        +-----------------------+
                        |   Linker Statistics   |
                        +-----------------------+

Stack size:  00016800 (92160.)
Memory size:  002d5b32 (2972466.)
Entry point address: 0001:00078c94
Link time: 00:00.35
